 jaccesswalker-32

 Timestamp is ffffffff (Sun Feb  7 06:28:15 2106)

 Preferred load address is 00400000

 Start         Length     Name                   Class
 0001:00000000 000070c0H .text$mn                CODE
 0001:000070c0 00000044H .text$x                 CODE
 0002:00000000 000001c4H .idata$5                DATA
 0002:000001c4 00000004H .00cfg                  DATA
 0002:000001c8 00000004H .CRT$XCA                DATA
 0002:000001cc 00000004H .CRT$XCAA               DATA
 0002:000001d0 00000004H .CRT$XCZ                DATA
 0002:000001d4 00000004H .CRT$XIA                DATA
 0002:000001d8 00000004H .CRT$XIAA               DATA
 0002:000001dc 00000004H .CRT$XIAC               DATA
 0002:000001e0 00000004H .CRT$XIZ                DATA
 0002:000001e4 00000004H .CRT$XPA                DATA
 0002:000001e8 00000004H .CRT$XPZ                DATA
 0002:000001ec 00000004H .CRT$XTA                DATA
 0002:000001f0 00000008H .CRT$XTZ                DATA
 0002:000001f4 00000000H .gfids$y                DATA
 0002:000001f8 00001a00H .rdata                  DATA
 0002:00001bf8 0000012cH .rdata$r                DATA
 0002:00001d24 00000008H .rdata$sxdata           DATA
 0002:00001d2c 000002f0H .rdata$zzzdbg           DATA
 0002:0000201c 00000004H .rtc$IAA                DATA
 0002:00002020 00000004H .rtc$IZZ                DATA
 0002:00002024 00000004H .rtc$TAA                DATA
 0002:00002028 00000008H .rtc$TZZ                DATA
 0002:00002030 000000fcH .xdata$x                DATA
 0002:0000212c 00000000H .edata                  DATA
 0002:0000212c 00000104H .idata$2                DATA
 0002:00002230 00000014H .idata$3                DATA
 0002:00002244 000001c4H .idata$4                DATA
 0002:00002408 0000083eH .idata$6                DATA
 0003:00000000 00000ae8H .data                   DATA
 0003:00000ae8 00000078H .data$r                 DATA
 0003:00000b60 00000690H .bss                    DATA
 0004:00000000 000001d0H .rsrc$01                DATA
 0004:000001d0 00000558H .rsrc$02                DATA

  Address         Publics by Value              Rva+Base       Lib:Object

 0000:00000000       ___x64_code_ranges_to_entry_points 00000000     <absolute>
 0000:00000000       ___guard_iat_table         00000000     <absolute>
 0000:00000000       ___arm64x_redirection_metadata_count 00000000     <absolute>
 0000:00000000       ___guard_fids_table        00000000     <absolute>
 0000:00000000       ___arm64x_extra_rfe_table  00000000     <absolute>
 0000:00000000       ___arm64x_native_entrypoint 00000000     <absolute>
 0000:00000000       ___hybrid_code_map         00000000     <absolute>
 0000:00000000       ___enclave_config          00000000     <absolute>
 0000:00000000       ___volatile_metadata       00000000     <absolute>
 0000:00000000       ___hybrid_auxiliary_iat    00000000     <absolute>
 0000:00000000       ___arm64x_extra_rfe_table_size 00000000     <absolute>
 0000:00000000       ___guard_longjmp_count     00000000     <absolute>
 0000:00000000       ___dynamic_value_reloc_table 00000000     <absolute>
 0000:00000000       ___guard_eh_cont_table     00000000     <absolute>
 0000:00000000       ___hybrid_code_map_count   00000000     <absolute>
 0000:00000000       ___AbsoluteZero            00000000     <absolute>
 0000:00000000       ___guard_longjmp_table     00000000     <absolute>
 0000:00000000       ___guard_fids_count        00000000     <absolute>
 0000:00000000       ___x64_code_ranges_to_entry_points_count 00000000     <absolute>
 0000:00000000       ___guard_iat_count         00000000     <absolute>
 0000:00000000       ___arm64x_redirection_metadata 00000000     <absolute>
 0000:00000000       ___guard_eh_cont_count     00000000     <absolute>
 0000:00000002       ___safe_se_handler_count   00000002     <absolute>
 0000:00000100       ___guard_flags             00000100     <absolute>
 0000:00000000       ___ImageBase               00400000     <linker-defined>
 0001:00000000       _initializeAccessBridge    00401000 f   AccessBridgeCalls.obj
 0001:00000ec0       _shutdownAccessBridge      00401ec0 f   AccessBridgeCalls.obj
 0001:00000f10       _IsJavaWindow              00401f10 f   AccessBridgeCalls.obj
 0001:00000f40       _GetAccessibleContextFromHWND 00401f40 f   AccessBridgeCalls.obj
 0001:00000f70       _getHWNDFromAccessibleContext 00401f70 f   AccessBridgeCalls.obj
 0001:00000fa0       _SetJavaShutdown           00401fa0 f   AccessBridgeCalls.obj
 0001:00000fc0       _SetFocusGained            00401fc0 f   AccessBridgeCalls.obj
 0001:00000fe0       _SetFocusLost              00401fe0 f   AccessBridgeCalls.obj
 0001:00001000       _SetCaretUpdate            00402000 f   AccessBridgeCalls.obj
 0001:00001020       _SetMouseClicked           00402020 f   AccessBridgeCalls.obj
 0001:00001040       _SetMouseEntered           00402040 f   AccessBridgeCalls.obj
 0001:00001060       _SetMouseExited            00402060 f   AccessBridgeCalls.obj
 0001:00001080       _SetMousePressed           00402080 f   AccessBridgeCalls.obj
 0001:000010a0       _SetMouseReleased          004020a0 f   AccessBridgeCalls.obj
 0001:000010c0       _SetMenuCanceled           004020c0 f   AccessBridgeCalls.obj
 0001:000010e0       _SetMenuDeselected         004020e0 f   AccessBridgeCalls.obj
 0001:00001100       _SetMenuSelected           00402100 f   AccessBridgeCalls.obj
 0001:00001120       _SetPopupMenuCanceled      00402120 f   AccessBridgeCalls.obj
 0001:00001140       _SetPopupMenuWillBecomeInvisible 00402140 f   AccessBridgeCalls.obj
 0001:00001160       _SetPopupMenuWillBecomeVisible 00402160 f   AccessBridgeCalls.obj
 0001:00001180       _SetPropertyNameChange     00402180 f   AccessBridgeCalls.obj
 0001:000011a0       _SetPropertyDescriptionChange 004021a0 f   AccessBridgeCalls.obj
 0001:000011c0       _SetPropertyStateChange    004021c0 f   AccessBridgeCalls.obj
 0001:000011e0       _SetPropertyValueChange    004021e0 f   AccessBridgeCalls.obj
 0001:00001200       _SetPropertySelectionChange 00402200 f   AccessBridgeCalls.obj
 0001:00001220       _SetPropertyTextChange     00402220 f   AccessBridgeCalls.obj
 0001:00001240       _SetPropertyCaretChange    00402240 f   AccessBridgeCalls.obj
 0001:00001260       _SetPropertyVisibleDataChange 00402260 f   AccessBridgeCalls.obj
 0001:00001280       _SetPropertyChildChange    00402280 f   AccessBridgeCalls.obj
 0001:000012a0       _SetPropertyActiveDescendentChange 004022a0 f   AccessBridgeCalls.obj
 0001:000012c0       _SetPropertyTableModelChange 004022c0 f   AccessBridgeCalls.obj
 0001:000012e0       _ReleaseJavaObject         004022e0 f   AccessBridgeCalls.obj
 0001:00001310       _GetVersionInfo            00402310 f   AccessBridgeCalls.obj
 0001:00001340       _GetAccessibleContextAt    00402340 f   AccessBridgeCalls.obj
 0001:00001380       _GetAccessibleContextWithFocus 00402380 f   AccessBridgeCalls.obj
 0001:000013b0       _GetAccessibleContextInfo  004023b0 f   AccessBridgeCalls.obj
 0001:000013e0       _GetAccessibleChildFromContext 004023e0 f   AccessBridgeCalls.obj
 0001:00001410       _GetAccessibleParentFromContext 00402410 f   AccessBridgeCalls.obj
 0001:00001440       _GetAccessibleTextInfo     00402440 f   AccessBridgeCalls.obj
 0001:00001480       _GetAccessibleTextItems    00402480 f   AccessBridgeCalls.obj
 0001:000014b0       _GetAccessibleTextSelectionInfo 004024b0 f   AccessBridgeCalls.obj
 0001:000014e0       _GetAccessibleTextAttributes 004024e0 f   AccessBridgeCalls.obj
 0001:00001510       _GetAccessibleTextRect     00402510 f   AccessBridgeCalls.obj
 0001:00001540       _GetAccessibleTextLineBounds 00402540 f   AccessBridgeCalls.obj
 0001:00001580       _GetAccessibleTextRange    00402580 f   AccessBridgeCalls.obj
 0001:000015c0       _getAccessibleTableInfo    004025c0 f   AccessBridgeCalls.obj
 0001:000015f0       _getAccessibleTableCellInfo 004025f0 f   AccessBridgeCalls.obj
 0001:00001630       _getAccessibleTableRowHeader 00402630 f   AccessBridgeCalls.obj
 0001:00001660       _getAccessibleTableColumnHeader 00402660 f   AccessBridgeCalls.obj
 0001:00001690       _getAccessibleTableRowDescription 00402690 f   AccessBridgeCalls.obj
 0001:000016c0       _getAccessibleTableColumnDescription 004026c0 f   AccessBridgeCalls.obj
 0001:000016f0       _getAccessibleTableRowSelectionCount 004026f0 f   AccessBridgeCalls.obj
 0001:00001720       _isAccessibleTableRowSelected 00402720 f   AccessBridgeCalls.obj
 0001:00001750       _getAccessibleTableRowSelections 00402750 f   AccessBridgeCalls.obj
 0001:00001780       _getAccessibleTableColumnSelectionCount 00402780 f   AccessBridgeCalls.obj
 0001:000017b0       _isAccessibleTableColumnSelected 004027b0 f   AccessBridgeCalls.obj
 0001:000017e0       _getAccessibleTableColumnSelections 004027e0 f   AccessBridgeCalls.obj
 0001:00001810       _getAccessibleTableRow     00402810 f   AccessBridgeCalls.obj
 0001:00001840       _getAccessibleTableColumn  00402840 f   AccessBridgeCalls.obj
 0001:00001870       _getAccessibleTableIndex   00402870 f   AccessBridgeCalls.obj
 0001:000018a0       _getAccessibleRelationSet  004028a0 f   AccessBridgeCalls.obj
 0001:000018d0       _getAccessibleHypertext    004028d0 f   AccessBridgeCalls.obj
 0001:00001900       _activateAccessibleHyperlink 00402900 f   AccessBridgeCalls.obj
 0001:00001930       _getAccessibleHyperlinkCount 00402930 f   AccessBridgeCalls.obj
 0001:00001960       _getAccessibleHypertextExt 00402960 f   AccessBridgeCalls.obj
 0001:00001990       _getAccessibleHypertextLinkIndex 00402990 f   AccessBridgeCalls.obj
 0001:000019c0       _getAccessibleHyperlink    004029c0 f   AccessBridgeCalls.obj
 0001:000019f0       _getAccessibleKeyBindings  004029f0 f   AccessBridgeCalls.obj
 0001:00001a20       _getAccessibleIcons        00402a20 f   AccessBridgeCalls.obj
 0001:00001a50       _getAccessibleActions      00402a50 f   AccessBridgeCalls.obj
 0001:00001a80       _doAccessibleActions       00402a80 f   AccessBridgeCalls.obj
 0001:00001ab0       _IsSameObject              00402ab0 f   AccessBridgeCalls.obj
 0001:00001ae0       _setTextContents           00402ae0 f   AccessBridgeCalls.obj
 0001:00001b10       _getParentWithRole         00402b10 f   AccessBridgeCalls.obj
 0001:00001b40       _getParentWithRoleElseRoot 00402b40 f   AccessBridgeCalls.obj
 0001:00001b70       _getTopLevelObject         00402b70 f   AccessBridgeCalls.obj
 0001:00001ba0       _getObjectDepth            00402ba0 f   AccessBridgeCalls.obj
 0001:00001bd0       _getActiveDescendent       00402bd0 f   AccessBridgeCalls.obj
 0001:00001c00       _GetCurrentAccessibleValueFromContext 00402c00 f   AccessBridgeCalls.obj
 0001:00001c30       _GetMaximumAccessibleValueFromContext 00402c30 f   AccessBridgeCalls.obj
 0001:00001c60       _GetMinimumAccessibleValueFromContext 00402c60 f   AccessBridgeCalls.obj
 0001:00001c90       _GetAccessibleSelectionFromContext 00402c90 f   AccessBridgeCalls.obj
 0001:00001cc0       _GetAccessibleSelectionCountFromContext 00402cc0 f   AccessBridgeCalls.obj
 0001:00001cf0       _IsAccessibleChildSelectedFromContext 00402cf0 f   AccessBridgeCalls.obj
 0001:00001d20       _RemoveAccessibleSelectionFromContext 00402d20 f   AccessBridgeCalls.obj
 0001:00001d50       _SelectAllAccessibleSelectionFromContext 00402d50 f   AccessBridgeCalls.obj
 0001:00001d80       _getVirtualAccessibleName  00402d80 f   AccessBridgeCalls.obj
 0001:00001db0       _requestFocus              00402db0 f   AccessBridgeCalls.obj
 0001:00001de0       _selectTextRange           00402de0 f   AccessBridgeCalls.obj
 0001:00001e10       _getTextAttributesInRange  00402e10 f   AccessBridgeCalls.obj
 0001:00001e50       _getVisibleChildrenCount   00402e50 f   AccessBridgeCalls.obj
 0001:00001e80       _getVisibleChildren        00402e80 f   AccessBridgeCalls.obj
 0001:00001eb0       _setCaretPosition          00402eb0 f   AccessBridgeCalls.obj
 0001:00001ee0       _getCaretLocation          00402ee0 f   AccessBridgeCalls.obj
 0001:00001f10       _getEventsWaiting          00402f10 f   AccessBridgeCalls.obj
 0001:00001f30       _addAccessibleSelectionFromContext 00402f30 f   AccessBridgeCalls.obj
 0001:00001f60       _clearAccessibleSelectionFromContext 00402f60 f   AccessBridgeCalls.obj
 0001:00001fa0       _printError                00402fa0 f   AccessBridgeDebug.obj
 0001:000020b0       _PrintDebugString          004030b0 f   AccessBridgeDebug.obj
 0001:00002120       _wPrintJavaDebugString     00403120 f   AccessBridgeDebug.obj
 0001:00002190       _wPrintDebugString         00403190 f   AccessBridgeDebug.obj
 0001:00002200       _initializeFileLogger      00403200 f   AccessBridgeDebug.obj
 0001:00002330       _finalizeFileLogger        00403330 f   AccessBridgeDebug.obj
 0001:00002360       _getTimeStamp              00403360 f   AccessBridgeDebug.obj
 0001:000023a0       _PrintJavaDebugString2     004033a0 f   AccessBridgeDebug.obj
 0001:00002410       ___local_stdio_printf_options 00403410 f i AccessBridgeDebug.obj
 0001:00002420       __vfprintf_l               00403420 f i AccessBridgeDebug.obj
 0001:00002450       __vfwprintf_l              00403450 f i AccessBridgeDebug.obj
 0001:00002480       _fprintf                   00403480 f i AccessBridgeDebug.obj
 0001:000024c0       _printf                    004034c0 f i AccessBridgeDebug.obj
 0001:00002500       _vfprintf                  00403500 f i AccessBridgeDebug.obj
 0001:00002520       _vfwprintf                 00403520 f i AccessBridgeDebug.obj
 0001:00002540       ?initBroadcastMessageIDs@@YAHXZ 00403540 f   AccessBridgeMessages.obj
 0001:00002580       ?getTimeAndDate@@YAPADXZ   00403580 f   AccessInfo.obj
 0001:00002630       ?displayAndLog@@YAXPAUHWND__@@HPAU_iobuf@@PADZZ 00403630 f   AccessInfo.obj
 0001:00002710       ?logString@@YAXPAU_iobuf@@PADZZ 00403710 f   AccessInfo.obj
 0001:000027a0       ?getAccessibleInfo@@YAPADJ_JPADH@Z 004037a0 f   AccessInfo.obj
 0001:000027d0       ?getAccessibleInfo@@YAPADJ_JHHPADH@Z 004037d0 f   AccessInfo.obj
 0001:000049d0       ?appendToBuffer@@YAHPADI0ZZ 004059d0 f   AccessInfo.obj
 0001:00004ab0       __vsnprintf_l              00405ab0 f i AccessInfo.obj
 0001:00004b10       __vsprintf_l               00405b10 f i AccessInfo.obj
 0001:00004b30       _sprintf                   00405b30 f i AccessInfo.obj
 0001:00004b70       _vsprintf                  00405b70 f i AccessInfo.obj
 0001:00004b90       _WinMain@16                00405b90 f   jaccesswalker.obj
 0001:00004c20       ??0AccessibleNode@@QAE@J_JPAV0@PAUHWND__@@PAU_TREEITEM@@@Z 00405c20 f   jaccesswalker.obj
 0001:00004c70       ??1AccessibleNode@@QAE@XZ  00405c70 f   jaccesswalker.obj
 0001:00004ca0       ?setAccessibleName@AccessibleNode@@QAEXPAD@Z 00405ca0 f   jaccesswalker.obj
 0001:00004cd0       ?setAccessibleRole@AccessibleNode@@QAEXPAD@Z 00405cd0 f   jaccesswalker.obj
 0001:00004d00       ?displayAPIWindow@AccessibleNode@@QAEHXZ 00405d00 f   jaccesswalker.obj
 0001:00004e30       ??0Jaccesswalker@@QAE@H@Z  00405e30 f   jaccesswalker.obj
 0001:00004ff0       ?buildAccessibilityTree@Jaccesswalker@@QAEXXZ 00405ff0 f   jaccesswalker.obj
 0001:00005020       ?addComponentNodes@Jaccesswalker@@QAEXJ_JPAVAccessibleNode@@PAUHWND__@@PAU_TREEITEM@@2@Z 00406020 f   jaccesswalker.obj
 0001:00005320       ?WinProc@@YGJPAUHWND__@@IIJ@Z 00406320 f   jaccesswalker.obj
 0001:000055f0       ?EnumWndProc@@YGHPAUHWND__@@J@Z 004065f0 f   jaccesswalker.obj
 0001:000056f0       ?EnumChildProc@@YGHPAUHWND__@@J@Z 004066f0 f   jaccesswalker.obj
 0001:00005790       ?CreateATreeView@@YAPAUHWND__@@PAU1@@Z 00406790 f   jaccesswalker.obj
 0001:00005800       ?AccessInfoWindowProc@@YGJPAUHWND__@@IIJ@Z 00406800 f   jaccesswalker.obj
 0001:00005900       ?IsInaccessibleJavaWindow@@YAHQAUHWND__@@@Z 00406900 f   jaccesswalker.obj
 0001:000060a9       ??_U@YAPAXI@Z              004070a9 f   MSVCRT:new_array.obj
 0001:000060b2       ??_V@YAXPAX@Z              004070b2 f   MSVCRT:delete_array.obj
 0001:000060b7       ___raise_securityfailure   004070b7 f   MSVCRT:gs_report.obj
 0001:000060df       ___report_gsfailure        004070df f   MSVCRT:gs_report.obj
 0001:000061d8       ___report_rangecheckfailure 004071d8 f   MSVCRT:gs_report.obj
 0001:000061e4       ___report_securityfailure  004071e4 f   MSVCRT:gs_report.obj
 0001:000062c0       __aulldiv                  004072c0 f   MSVCRT:ulldiv.obj
 0001:00006328       @__security_check_cookie@4 00407328 f   MSVCRT:secchk.obj
 0001:00006340       __alloca_probe             00407340 f   MSVCRT:chkstk.obj
 0001:00006340       __chkstk                   00407340 f   MSVCRT:chkstk.obj
 0001:0000636d       ??2@YAPAXI@Z               0040736d f   MSVCRT:new_scalar.obj
 0001:0000639d       ??3@YAXPAXI@Z              0040739d f   MSVCRT:delete_scalar_size.obj
 0001:000065ec       _WinMainCRTStartup         004075ec f   MSVCRT:exe_winmain.obj
 0001:000065f6       ??3@YAXPAX@Z               004075f6 f   MSVCRT:delete_scalar.obj
 0001:000065fb       ??0bad_alloc@std@@QAE@ABV01@@Z 004075fb f i MSVCRT:throw_bad_alloc.obj
 0001:00006616       ??0bad_alloc@std@@QAE@XZ   00407616 f i MSVCRT:throw_bad_alloc.obj
 0001:0000662e       ??0bad_array_new_length@std@@QAE@ABV01@@Z 0040762e f i MSVCRT:throw_bad_alloc.obj
 0001:00006649       ??0bad_array_new_length@std@@QAE@XZ 00407649 f i MSVCRT:throw_bad_alloc.obj
 0001:00006661       ??0exception@std@@QAE@ABV01@@Z 00407661 f i MSVCRT:throw_bad_alloc.obj
 0001:0000668d       ??1bad_alloc@std@@UAE@XZ   0040768d f i MSVCRT:throw_bad_alloc.obj
 0001:0000668d       ??1bad_array_new_length@std@@UAE@XZ 0040768d f i MSVCRT:throw_bad_alloc.obj
 0001:0000669e       ??_Gexception@std@@UAEPAXI@Z 0040769e f i MSVCRT:throw_bad_alloc.obj
 0001:0000669e       ??_Ebad_array_new_length@std@@UAEPAXI@Z 0040769e f i MSVCRT:throw_bad_alloc.obj
 0001:0000669e       ??_Gbad_alloc@std@@UAEPAXI@Z 0040769e f i MSVCRT:throw_bad_alloc.obj
 0001:0000669e       ??_Ebad_alloc@std@@UAEPAXI@Z 0040769e f i MSVCRT:throw_bad_alloc.obj
 0001:0000669e       ??_Gbad_array_new_length@std@@UAEPAXI@Z 0040769e f i MSVCRT:throw_bad_alloc.obj
 0001:0000669e       ??_Eexception@std@@UAEPAXI@Z 0040769e f i MSVCRT:throw_bad_alloc.obj
 0001:000066cb       ?__scrt_throw_std_bad_alloc@@YAXXZ 004076cb f   MSVCRT:throw_bad_alloc.obj
 0001:000066e8       ?__scrt_throw_std_bad_array_new_length@@YAXXZ 004076e8 f   MSVCRT:throw_bad_alloc.obj
 0001:00006705       ?what@exception@std@@UBEPBDXZ 00407705 f i MSVCRT:throw_bad_alloc.obj
 0001:00006756       ___scrt_acquire_startup_lock 00407756 f   MSVCRT:utility.obj
 0001:00006788       ___scrt_initialize_crt     00407788 f   MSVCRT:utility.obj
 0001:000067c1       ___scrt_initialize_onexit_tables 004077c1 f   MSVCRT:utility.obj
 0001:00006848       ___scrt_is_nonwritable_in_current_image 00407848 f   MSVCRT:utility.obj
 0001:000068dc       ___scrt_release_startup_lock 004078dc f   MSVCRT:utility.obj
 0001:000068f9       ___scrt_uninitialize_crt   004078f9 f   MSVCRT:utility.obj
 0001:00006921       __onexit                   00407921 f   MSVCRT:utility.obj
 0001:0000694e       _atexit                    0040794e f   MSVCRT:utility.obj
 0001:000069b0       ___security_init_cookie    004079b0 f   MSVCRT:gs_support.obj
 0001:000069fb       __get_startup_new_mode     004079fb f   MSVCRT:new_mode.obj
 0001:000069fb       __matherr                  004079fb f   MSVCRT:matherr.obj
 0001:000069fb       ___scrt_initialize_winrt   004079fb f   MSVCRT:utility_desktop.obj
 0001:000069fb       __get_startup_commit_mode  004079fb f   MSVCRT:commit_mode.obj
 0001:000069fb       ___scrt_stub_for_initialize_mta 004079fb f   MSVCRT:utility_desktop.obj
 0001:000069fb       __get_startup_thread_locale_mode 004079fb f   MSVCRT:thread_locale.obj
 0001:000069fb       ___scrt_exe_initialize_mta 004079fb f   MSVCRT:utility_desktop.obj
 0001:000069fe       __get_startup_argv_mode    004079fe f   MSVCRT:argv_mode.obj
 0001:00006a02       __get_startup_file_mode    00407a02 f   MSVCRT:file_mode.obj
 0001:00006a08       ?__scrt_initialize_type_info@@YAXXZ 00407a08 f   MSVCRT:tncleanup.obj
 0001:00006a14       ___acrt_uninitialize       00407a14 f   MSVCRT:ucrt_stubs.obj
 0001:00006a14       ___scrt_stub_for_acrt_initialize 00407a14 f   MSVCRT:ucrt_stubs.obj
 0001:00006a14       ___scrt_stub_for_acrt_uninitialize 00407a14 f   MSVCRT:ucrt_stubs.obj
 0001:00006a14       ___acrt_initialize         00407a14 f   MSVCRT:ucrt_stubs.obj
 0001:00006a14       ___vcrt_uninitialize       00407a14 f   MSVCRT:ucrt_stubs.obj
 0001:00006a14       ___vcrt_initialize         00407a14 f   MSVCRT:ucrt_stubs.obj
 0001:00006a14       __should_initialize_environment 00407a14 f   MSVCRT:env_mode.obj
 0001:00006a17       __initialize_default_precision 00407a17 f   MSVCRT:default_precision.obj
 0001:00006a38       @_guard_check_icall_nop@4  00407a38 f   MSVCRT:guard_support.obj
 0001:00006a38       __initialize_invalid_parameter_handler 00407a38 f   MSVCRT:invalid_parameter_handler.obj
 0001:00006a38       __initialize_denormal_control 00407a38 f   MSVCRT:denormal_control.obj
 0001:00006a3b       ___local_stdio_scanf_options 00407a3b f i MSVCRT:default_local_stdio_options.obj
 0001:00006a41       ___scrt_initialize_default_local_stdio_options 00407a41 f   MSVCRT:default_local_stdio_options.obj
 0001:00006a5e       ___scrt_is_user_matherr_present 00407a5e f   MSVCRT:matherr_detection.obj
 0001:00006a6a       ___scrt_get_dyn_tls_init_callback 00407a6a f   MSVCRT:dyn_tls_init.obj
 0001:00006a70       ___scrt_get_dyn_tls_dtor_callback 00407a70 f   MSVCRT:dyn_tls_dtor.obj
 0001:00006a76       ___scrt_fastfail           00407a76 f   MSVCRT:utility_desktop.obj
 0001:00006b90       ___scrt_get_show_window_mode 00407b90 f   MSVCRT:utility_desktop.obj
 0001:00006bc1       ___scrt_initialize_mta     00407bc1 f   MSVCRT:utility_desktop.obj
 0001:00006bc6       ___scrt_is_managed_app     00407bc6 f   MSVCRT:utility_desktop.obj
 0001:00006c09       ___scrt_set_unhandled_exception_filter 00407c09 f   MSVCRT:utility_desktop.obj
 0001:00006c15       ___scrt_unhandled_exception_filter@4 00407c15 f   MSVCRT:utility_desktop.obj
 0001:00006c6b       __crt_debugger_hook        00407c6b f   MSVCRT:utility_desktop.obj
 0001:00006c73       __RTC_Initialize           00407c73 f   MSVCRT:initsect.obj
 0001:00006c9f       __RTC_Terminate            00407c9f f   MSVCRT:initsect.obj
 0001:00006cd0       __SEH_prolog4              00407cd0 f   MSVCRT:sehprolg4.obj
 0001:00006d14       __SEH_epilog4              00407d14 f   MSVCRT:sehprolg4.obj
 0001:00006d28       __except_handler4          00407d28 f   MSVCRT:chandler4gs.obj
 0001:00006d57       ??_Gtype_info@@UAEPAXI@Z   00407d57 f i MSVCRT:std_type_info_static.obj
 0001:00006d57       ??_Etype_info@@UAEPAXI@Z   00407d57 f i MSVCRT:std_type_info_static.obj
 0001:00006d7a       ___isa_available_init      00407d7a f   MSVCRT:cpu_disp.obj
 0001:00006f4a       ___scrt_is_ucrt_dll_in_use 00407f4a f   MSVCRT:ucrt_detection.obj
 0001:00006f56       _IsProcessorFeaturePresent@4 00407f56 f   kernel32:KERNEL32.dll
 0001:00006f5c       _memcpy                    00407f5c f   vcruntime:VCRUNTIME140.dll
 0001:00006f62       _memset                    00407f62 f   vcruntime:VCRUNTIME140.dll
 0001:00006f68       ___CxxFrameHandler3        00407f68 f   vcruntime:VCRUNTIME140.dll
 0001:00006f6e       ___std_exception_copy      00407f6e f   vcruntime:VCRUNTIME140.dll
 0001:00006f74       ___std_exception_destroy   00407f74 f   vcruntime:VCRUNTIME140.dll
 0001:00006f7a       __CxxThrowException@8      00407f7a f   vcruntime:VCRUNTIME140.dll
 0001:00006f80       ___current_exception       00407f80 f   vcruntime:VCRUNTIME140.dll
 0001:00006f86       ___current_exception_context 00407f86 f   vcruntime:VCRUNTIME140.dll
 0001:00006f8c       __except_handler4_common   00407f8c f   vcruntime:VCRUNTIME140.dll
 0001:00006f92       _strlen                    00407f92 f   ucrt:api-ms-win-crt-string-l1-1-0.dll
 0001:00006f98       _strcpy                    00407f98 f   ucrt:api-ms-win-crt-string-l1-1-0.dll
 0001:00006f9e       _strcmp                    00407f9e f   ucrt:api-ms-win-crt-string-l1-1-0.dll
 0001:00006fa4       __callnewh                 00407fa4 f   ucrt:api-ms-win-crt-heap-l1-1-0.dll
 0001:00006faa       _malloc                    00407faa f   ucrt:api-ms-win-crt-heap-l1-1-0.dll
 0001:00006fb0       __seh_filter_exe           00407fb0 f   ucrt:api-ms-win-crt-runtime-l1-1-0.dll
 0001:00006fb6       __set_app_type             00407fb6 f   ucrt:api-ms-win-crt-runtime-l1-1-0.dll
 0001:00006fbc       ___setusermatherr          00407fbc f   ucrt:api-ms-win-crt-math-l1-1-0.dll
 0001:00006fc2       __configure_narrow_argv    00407fc2 f   ucrt:api-ms-win-crt-runtime-l1-1-0.dll
 0001:00006fc8       __initialize_narrow_environment 00407fc8 f   ucrt:api-ms-win-crt-runtime-l1-1-0.dll
 0001:00006fce       __get_narrow_winmain_command_line 00407fce f   ucrt:api-ms-win-crt-runtime-l1-1-0.dll
 0001:00006fd4       __initterm                 00407fd4 f   ucrt:api-ms-win-crt-runtime-l1-1-0.dll
 0001:00006fda       __initterm_e               00407fda f   ucrt:api-ms-win-crt-runtime-l1-1-0.dll
 0001:00006fe0       _exit                      00407fe0 f   ucrt:api-ms-win-crt-runtime-l1-1-0.dll
 0001:00006fe6       __exit                     00407fe6 f   ucrt:api-ms-win-crt-runtime-l1-1-0.dll
 0001:00006fec       __set_fmode                00407fec f   ucrt:api-ms-win-crt-stdio-l1-1-0.dll
 0001:00006ff2       __cexit                    00407ff2 f   ucrt:api-ms-win-crt-runtime-l1-1-0.dll
 0001:00006ff8       __c_exit                   00407ff8 f   ucrt:api-ms-win-crt-runtime-l1-1-0.dll
 0001:00006ffe       __register_thread_local_exe_atexit_callback 00407ffe f   ucrt:api-ms-win-crt-runtime-l1-1-0.dll
 0001:00007004       __configthreadlocale       00408004 f   ucrt:api-ms-win-crt-locale-l1-1-0.dll
 0001:0000700a       __set_new_mode             0040800a f   ucrt:api-ms-win-crt-heap-l1-1-0.dll
 0001:00007010       ___p__commode              00408010 f   ucrt:api-ms-win-crt-stdio-l1-1-0.dll
 0001:00007016       _free                      00408016 f   ucrt:api-ms-win-crt-heap-l1-1-0.dll
 0001:0000701c       __initialize_onexit_table  0040801c f   ucrt:api-ms-win-crt-runtime-l1-1-0.dll
 0001:00007022       __register_onexit_function 00408022 f   ucrt:api-ms-win-crt-runtime-l1-1-0.dll
 0001:00007028       __crt_atexit               00408028 f   ucrt:api-ms-win-crt-runtime-l1-1-0.dll
 0001:0000702e       __controlfp_s              0040802e f   ucrt:api-ms-win-crt-runtime-l1-1-0.dll
 0001:00007034       _terminate                 00408034 f   ucrt:api-ms-win-crt-runtime-l1-1-0.dll
 0001:0000703a       __filter_x86_sse2_floating_point_exception 0040803a f   MSVCRT:x86_exception_filter.obj
 0001:0000703a       __filter_x86_sse2_floating_point_exception_default 0040803a f   MSVCRT:x86_exception_filter.obj
 0002:00000000       __imp__InitCommonControlsEx@4 00409000     comctl32:COMCTL32.dll
 0002:00000004       \177COMCTL32_NULL_THUNK_DATA 00409004     comctl32:COMCTL32.dll
 0002:00000008       __imp__GetStockObject@4    00409008     gdi32:GDI32.dll
 0002:0000000c       \177GDI32_NULL_THUNK_DATA  0040900c     gdi32:GDI32.dll
 0002:00000010       __imp__GetModuleHandleW@4  00409010     kernel32:KERNEL32.dll
 0002:00000014       __imp__GetStartupInfoW@4   00409014     kernel32:KERNEL32.dll
 0002:00000018       __imp__IsDebuggerPresent@0 00409018     kernel32:KERNEL32.dll
 0002:0000001c       __imp__InitializeSListHead@4 0040901c     kernel32:KERNEL32.dll
 0002:00000020       __imp__GetCurrentThreadId@0 00409020     kernel32:KERNEL32.dll
 0002:00000024       __imp__GetCurrentProcessId@0 00409024     kernel32:KERNEL32.dll
 0002:00000028       __imp__QueryPerformanceCounter@4 00409028     kernel32:KERNEL32.dll
 0002:0000002c       __imp__IsProcessorFeaturePresent@4 0040902c     kernel32:KERNEL32.dll
 0002:00000030       __imp__TerminateProcess@8  00409030     kernel32:KERNEL32.dll
 0002:00000034       __imp__GetCurrentProcess@0 00409034     kernel32:KERNEL32.dll
 0002:00000038       __imp__SetUnhandledExceptionFilter@4 00409038     kernel32:KERNEL32.dll
 0002:0000003c       __imp__UnhandledExceptionFilter@4 0040903c     kernel32:KERNEL32.dll
 0002:00000040       __imp__FormatMessageA@28   00409040     kernel32:KERNEL32.dll
 0002:00000044       __imp__LocalFree@4         00409044     kernel32:KERNEL32.dll
 0002:00000048       __imp__GetSystemTimeAsFileTime@4 00409048     kernel32:KERNEL32.dll
 0002:0000004c       __imp__LoadLibraryA@4      0040904c     kernel32:KERNEL32.dll
 0002:00000050       __imp__GetProcAddress@8    00409050     kernel32:KERNEL32.dll
 0002:00000054       __imp__FreeLibrary@4       00409054     kernel32:KERNEL32.dll
 0002:00000058       __imp__GetLastError@0      00409058     kernel32:KERNEL32.dll
 0002:0000005c       \177KERNEL32_NULL_THUNK_DATA 0040905c     kernel32:KERNEL32.dll
 0002:00000060       __imp__GetClientRect@8     00409060     user32:USER32.dll
 0002:00000064       __imp__GetCursorPos@4      00409064     user32:USER32.dll
 0002:00000068       __imp__UpdateWindow@4      00409068     user32:USER32.dll
 0002:0000006c       __imp__EnumChildWindows@12 0040906c     user32:USER32.dll
 0002:00000070       __imp__EnumWindows@8       00409070     user32:USER32.dll
 0002:00000074       __imp__GetClassNameA@12    00409074     user32:USER32.dll
 0002:00000078       __imp__LoadCursorA@8       00409078     user32:USER32.dll
 0002:0000007c       __imp__LoadIconA@8         0040907c     user32:USER32.dll
 0002:00000080       __imp__RegisterWindowMessageA@4 00409080     user32:USER32.dll
 0002:00000084       __imp__TrackPopupMenu@28   00409084     user32:USER32.dll
 0002:00000088       __imp__GetSubMenu@8        00409088     user32:USER32.dll
 0002:0000008c       __imp__LoadMenuA@8         0040908c     user32:USER32.dll
 0002:00000090       __imp__GetDlgItem@8        00409090     user32:USER32.dll
 0002:00000094       __imp__EndDialog@8         00409094     user32:USER32.dll
 0002:00000098       __imp__SetWindowPos@28     00409098     user32:USER32.dll
 0002:0000009c       __imp__ShowWindow@8        0040909c     user32:USER32.dll
 0002:000000a0       __imp__DestroyWindow@4     004090a0     user32:USER32.dll
 0002:000000a4       __imp__CreateWindowExA@48  004090a4     user32:USER32.dll
 0002:000000a8       __imp__RegisterClassExA@4  004090a8     user32:USER32.dll
 0002:000000ac       __imp__PostQuitMessage@4   004090ac     user32:USER32.dll
 0002:000000b0       __imp__DefWindowProcA@16   004090b0     user32:USER32.dll
 0002:000000b4       __imp__SendMessageA@16     004090b4     user32:USER32.dll
 0002:000000b8       __imp__DispatchMessageA@4  004090b8     user32:USER32.dll
 0002:000000bc       __imp__TranslateMessage@4  004090bc     user32:USER32.dll
 0002:000000c0       __imp__GetMessageA@16      004090c0     user32:USER32.dll
 0002:000000c4       __imp__wsprintfA           004090c4     user32:USER32.dll
 0002:000000c8       __imp__SetDlgItemTextA@12  004090c8     user32:USER32.dll
 0002:000000cc       __imp__ScreenToClient@8    004090cc     user32:USER32.dll
 0002:000000d0       \177USER32_NULL_THUNK_DATA 004090d0     user32:USER32.dll
 0002:000000d4       __imp__memcpy              004090d4     vcruntime:VCRUNTIME140.dll
 0002:000000d8       __imp__memset              004090d8     vcruntime:VCRUNTIME140.dll
 0002:000000dc       __imp____CxxFrameHandler3  004090dc     vcruntime:VCRUNTIME140.dll
 0002:000000e0       __imp____std_exception_copy 004090e0     vcruntime:VCRUNTIME140.dll
 0002:000000e4       __imp____std_exception_destroy 004090e4     vcruntime:VCRUNTIME140.dll
 0002:000000e8       __imp___CxxThrowException@8 004090e8     vcruntime:VCRUNTIME140.dll
 0002:000000ec       __imp____current_exception 004090ec     vcruntime:VCRUNTIME140.dll
 0002:000000f0       __imp____current_exception_context 004090f0     vcruntime:VCRUNTIME140.dll
 0002:000000f4       __imp___except_handler4_common 004090f4     vcruntime:VCRUNTIME140.dll
 0002:000000f8       \177VCRUNTIME140_NULL_THUNK_DATA 004090f8     vcruntime:VCRUNTIME140.dll
 0002:000000fc       __imp__getenv              004090fc     ucrt:api-ms-win-crt-environment-l1-1-0.dll
 0002:00000100       \177api-ms-win-crt-environment-l1-1-0_NULL_THUNK_DATA 00409100     ucrt:api-ms-win-crt-environment-l1-1-0.dll
 0002:00000104       __imp___set_new_mode       00409104     ucrt:api-ms-win-crt-heap-l1-1-0.dll
 0002:00000108       __imp__malloc              00409108     ucrt:api-ms-win-crt-heap-l1-1-0.dll
 0002:0000010c       __imp___callnewh           0040910c     ucrt:api-ms-win-crt-heap-l1-1-0.dll
 0002:00000110       __imp__free                00409110     ucrt:api-ms-win-crt-heap-l1-1-0.dll
 0002:00000114       \177api-ms-win-crt-heap-l1-1-0_NULL_THUNK_DATA 00409114     ucrt:api-ms-win-crt-heap-l1-1-0.dll
 0002:00000118       __imp___configthreadlocale 00409118     ucrt:api-ms-win-crt-locale-l1-1-0.dll
 0002:0000011c       \177api-ms-win-crt-locale-l1-1-0_NULL_THUNK_DATA 0040911c     ucrt:api-ms-win-crt-locale-l1-1-0.dll
 0002:00000120       __imp____setusermatherr    00409120     ucrt:api-ms-win-crt-math-l1-1-0.dll
 0002:00000124       \177api-ms-win-crt-math-l1-1-0_NULL_THUNK_DATA 00409124     ucrt:api-ms-win-crt-math-l1-1-0.dll
 0002:00000128       __imp__terminate           00409128     ucrt:api-ms-win-crt-runtime-l1-1-0.dll
 0002:0000012c       __imp___controlfp_s        0040912c     ucrt:api-ms-win-crt-runtime-l1-1-0.dll
 0002:00000130       __imp___crt_atexit         00409130     ucrt:api-ms-win-crt-runtime-l1-1-0.dll
 0002:00000134       __imp___register_onexit_function 00409134     ucrt:api-ms-win-crt-runtime-l1-1-0.dll
 0002:00000138       __imp___initialize_onexit_table 00409138     ucrt:api-ms-win-crt-runtime-l1-1-0.dll
 0002:0000013c       __imp___seh_filter_exe     0040913c     ucrt:api-ms-win-crt-runtime-l1-1-0.dll
 0002:00000140       __imp___set_app_type       00409140     ucrt:api-ms-win-crt-runtime-l1-1-0.dll
 0002:00000144       __imp___c_exit             00409144     ucrt:api-ms-win-crt-runtime-l1-1-0.dll
 0002:00000148       __imp___configure_narrow_argv 00409148     ucrt:api-ms-win-crt-runtime-l1-1-0.dll
 0002:0000014c       __imp___initialize_narrow_environment 0040914c     ucrt:api-ms-win-crt-runtime-l1-1-0.dll
 0002:00000150       __imp___get_narrow_winmain_command_line 00409150     ucrt:api-ms-win-crt-runtime-l1-1-0.dll
 0002:00000154       __imp___initterm           00409154     ucrt:api-ms-win-crt-runtime-l1-1-0.dll
 0002:00000158       __imp___register_thread_local_exe_atexit_callback 00409158     ucrt:api-ms-win-crt-runtime-l1-1-0.dll
 0002:0000015c       __imp__exit                0040915c     ucrt:api-ms-win-crt-runtime-l1-1-0.dll
 0002:00000160       __imp___exit               00409160     ucrt:api-ms-win-crt-runtime-l1-1-0.dll
 0002:00000164       __imp___initterm_e         00409164     ucrt:api-ms-win-crt-runtime-l1-1-0.dll
 0002:00000168       __imp___cexit              00409168     ucrt:api-ms-win-crt-runtime-l1-1-0.dll
 0002:0000016c       \177api-ms-win-crt-runtime-l1-1-0_NULL_THUNK_DATA 0040916c     ucrt:api-ms-win-crt-runtime-l1-1-0.dll
 0002:00000170       __imp__fclose              00409170     ucrt:api-ms-win-crt-stdio-l1-1-0.dll
 0002:00000174       __imp____stdio_common_vfwprintf 00409174     ucrt:api-ms-win-crt-stdio-l1-1-0.dll
 0002:00000178       __imp____acrt_iob_func     00409178     ucrt:api-ms-win-crt-stdio-l1-1-0.dll
 0002:0000017c       __imp____p__commode        0040917c     ucrt:api-ms-win-crt-stdio-l1-1-0.dll
 0002:00000180       __imp____stdio_common_vsprintf 00409180     ucrt:api-ms-win-crt-stdio-l1-1-0.dll
 0002:00000184       __imp__fopen               00409184     ucrt:api-ms-win-crt-stdio-l1-1-0.dll
 0002:00000188       __imp____stdio_common_vfprintf 00409188     ucrt:api-ms-win-crt-stdio-l1-1-0.dll
 0002:0000018c       __imp___set_fmode          0040918c     ucrt:api-ms-win-crt-stdio-l1-1-0.dll
 0002:00000190       __imp__fflush              00409190     ucrt:api-ms-win-crt-stdio-l1-1-0.dll
 0002:00000194       \177api-ms-win-crt-stdio-l1-1-0_NULL_THUNK_DATA 00409194     ucrt:api-ms-win-crt-stdio-l1-1-0.dll
 0002:00000198       __imp__wcscmp              00409198     ucrt:api-ms-win-crt-string-l1-1-0.dll
 0002:0000019c       __imp__strncpy             0040919c     ucrt:api-ms-win-crt-string-l1-1-0.dll
 0002:000001a0       __imp__strlen              004091a0     ucrt:api-ms-win-crt-string-l1-1-0.dll
 0002:000001a4       __imp__strcmp              004091a4     ucrt:api-ms-win-crt-string-l1-1-0.dll
 0002:000001a8       __imp__strcpy              004091a8     ucrt:api-ms-win-crt-string-l1-1-0.dll
 0002:000001ac       __imp__strncat             004091ac     ucrt:api-ms-win-crt-string-l1-1-0.dll
 0002:000001b0       \177api-ms-win-crt-string-l1-1-0_NULL_THUNK_DATA 004091b0     ucrt:api-ms-win-crt-string-l1-1-0.dll
 0002:000001b4       __imp__asctime             004091b4     ucrt:api-ms-win-crt-time-l1-1-0.dll
 0002:000001b8       __imp___time64             004091b8     ucrt:api-ms-win-crt-time-l1-1-0.dll
 0002:000001bc       __imp___localtime64        004091bc     ucrt:api-ms-win-crt-time-l1-1-0.dll
 0002:000001c0       \177api-ms-win-crt-time-l1-1-0_NULL_THUNK_DATA 004091c0     ucrt:api-ms-win-crt-time-l1-1-0.dll
 0002:000001c4       ___guard_check_icall_fptr  004091c4     MSVCRT:guard_support.obj
 0002:000001c8       ___xc_a                    004091c8     MSVCRT:initializers.obj
 0002:000001d0       ___xc_z                    004091d0     MSVCRT:initializers.obj
 0002:000001d4       ___xi_a                    004091d4     MSVCRT:initializers.obj
 0002:000001e0       ___xi_z                    004091e0     MSVCRT:initializers.obj
 0002:000001e4       ___xp_a                    004091e4     MSVCRT:initializers.obj
 0002:000001e8       ___xp_z                    004091e8     MSVCRT:initializers.obj
 0002:000001ec       ___xt_a                    004091ec     MSVCRT:initializers.obj
 0002:000001f0       ___xt_z                    004091f0     MSVCRT:initializers.obj
 0002:00001a68       ??_7exception@std@@6B@     0040aa68     MSVCRT:throw_bad_alloc.obj
 0002:00001a70       ??_C@_0BC@EOODALEL@Unknown?5exception@ 0040aa70     MSVCRT:throw_bad_alloc.obj
 0002:00001a88       ??_7bad_alloc@std@@6B@     0040aa88     MSVCRT:throw_bad_alloc.obj
 0002:00001a90       ??_C@_0P@GHFPNOJB@bad?5allocation@ 0040aa90     MSVCRT:throw_bad_alloc.obj
 0002:00001aa4       ??_7bad_array_new_length@std@@6B@ 0040aaa4     MSVCRT:throw_bad_alloc.obj
 0002:00001aac       ??_C@_0BF@KINCDENJ@bad?5array?5new?5length@ 0040aaac     MSVCRT:throw_bad_alloc.obj
 0002:00001ac8       ??_7type_info@@6B@         0040aac8     MSVCRT:std_type_info_static.obj
 0002:00001b40       __load_config_used         0040ab40     MSVCRT:loadcfg.obj
 0002:00001bf8       ??_R4exception@std@@6B@    0040abf8     MSVCRT:throw_bad_alloc.obj
 0002:00001c0c       ??_R3exception@std@@8      0040ac0c     MSVCRT:throw_bad_alloc.obj
 0002:00001c1c       ??_R2exception@std@@8      0040ac1c     MSVCRT:throw_bad_alloc.obj
 0002:00001c24       ??_R1A@?0A@EA@exception@std@@8 0040ac24     MSVCRT:throw_bad_alloc.obj
 0002:00001c40       ??_R4bad_alloc@std@@6B@    0040ac40     MSVCRT:throw_bad_alloc.obj
 0002:00001c54       ??_R3bad_alloc@std@@8      0040ac54     MSVCRT:throw_bad_alloc.obj
 0002:00001c64       ??_R2bad_alloc@std@@8      0040ac64     MSVCRT:throw_bad_alloc.obj
 0002:00001c70       ??_R1A@?0A@EA@bad_alloc@std@@8 0040ac70     MSVCRT:throw_bad_alloc.obj
 0002:00001c8c       ??_R4bad_array_new_length@std@@6B@ 0040ac8c     MSVCRT:throw_bad_alloc.obj
 0002:00001ca0       ??_R3bad_array_new_length@std@@8 0040aca0     MSVCRT:throw_bad_alloc.obj
 0002:00001cb0       ??_R2bad_array_new_length@std@@8 0040acb0     MSVCRT:throw_bad_alloc.obj
 0002:00001cc0       ??_R1A@?0A@EA@bad_array_new_length@std@@8 0040acc0     MSVCRT:throw_bad_alloc.obj
 0002:00001cdc       ??_R4type_info@@6B@        0040acdc     MSVCRT:std_type_info_static.obj
 0002:00001cf0       ??_R3type_info@@8          0040acf0     MSVCRT:std_type_info_static.obj
 0002:00001d00       ??_R2type_info@@8          0040ad00     MSVCRT:std_type_info_static.obj
 0002:00001d08       ??_R1A@?0A@EA@type_info@@8 0040ad08     MSVCRT:std_type_info_static.obj
 0002:00001d24       ___safe_se_handler_table   0040ad24     <linker-defined>
 0002:0000201c       ___rtc_iaa                 0040b01c     MSVCRT:initsect.obj
 0002:00002020       ___rtc_izz                 0040b020     MSVCRT:initsect.obj
 0002:00002024       ___rtc_taa                 0040b024     MSVCRT:initsect.obj
 0002:00002028       ___rtc_tzz                 0040b028     MSVCRT:initsect.obj
 0002:0000207c       __TI2?AVbad_alloc@std@@    0040b07c     MSVCRT:throw_bad_alloc.obj
 0002:0000208c       __CTA2?AVbad_alloc@std@@   0040b08c     MSVCRT:throw_bad_alloc.obj
 0002:00002098       __CT??_R0?AVbad_alloc@std@@@8??0bad_alloc@std@@QAE@ABV01@@Z12 0040b098     MSVCRT:throw_bad_alloc.obj
 0002:000020b4       __CT??_R0?AVexception@std@@@8??0exception@std@@QAE@ABV01@@Z12 0040b0b4     MSVCRT:throw_bad_alloc.obj
 0002:000020d0       __TI3?AVbad_array_new_length@std@@ 0040b0d0     MSVCRT:throw_bad_alloc.obj
 0002:000020e0       __CTA3?AVbad_array_new_length@std@@ 0040b0e0     MSVCRT:throw_bad_alloc.obj
 0002:000020f0       __CT??_R0?AVbad_array_new_length@std@@@8??0bad_array_new_length@std@@QAE@ABV01@@Z12 0040b0f0     MSVCRT:throw_bad_alloc.obj
 0002:0000212c       __IMPORT_DESCRIPTOR_COMCTL32 0040b12c     comctl32:COMCTL32.dll
 0002:00002140       __IMPORT_DESCRIPTOR_GDI32  0040b140     gdi32:GDI32.dll
 0002:00002154       __IMPORT_DESCRIPTOR_USER32 0040b154     user32:USER32.dll
 0002:00002168       __IMPORT_DESCRIPTOR_KERNEL32 0040b168     kernel32:KERNEL32.dll
 0002:0000217c       __IMPORT_DESCRIPTOR_VCRUNTIME140 0040b17c     vcruntime:VCRUNTIME140.dll
 0002:00002190       __IMPORT_DESCRIPTOR_api-ms-win-crt-string-l1-1-0 0040b190     ucrt:api-ms-win-crt-string-l1-1-0.dll
 0002:000021a4       __IMPORT_DESCRIPTOR_api-ms-win-crt-stdio-l1-1-0 0040b1a4     ucrt:api-ms-win-crt-stdio-l1-1-0.dll
 0002:000021b8       __IMPORT_DESCRIPTOR_api-ms-win-crt-environment-l1-1-0 0040b1b8     ucrt:api-ms-win-crt-environment-l1-1-0.dll
 0002:000021cc       __IMPORT_DESCRIPTOR_api-ms-win-crt-time-l1-1-0 0040b1cc     ucrt:api-ms-win-crt-time-l1-1-0.dll
 0002:000021e0       __IMPORT_DESCRIPTOR_api-ms-win-crt-heap-l1-1-0 0040b1e0     ucrt:api-ms-win-crt-heap-l1-1-0.dll
 0002:000021f4       __IMPORT_DESCRIPTOR_api-ms-win-crt-runtime-l1-1-0 0040b1f4     ucrt:api-ms-win-crt-runtime-l1-1-0.dll
 0002:00002208       __IMPORT_DESCRIPTOR_api-ms-win-crt-math-l1-1-0 0040b208     ucrt:api-ms-win-crt-math-l1-1-0.dll
 0002:0000221c       __IMPORT_DESCRIPTOR_api-ms-win-crt-locale-l1-1-0 0040b21c     ucrt:api-ms-win-crt-locale-l1-1-0.dll
 0002:00002230       __NULL_IMPORT_DESCRIPTOR   0040b230     comctl32:COMCTL32.dll
 0003:00000a68       ?depth@@3HA                0040ca68     jaccesswalker.obj
 0003:00000a6c       ?theJaccesswalkerClassName@@3PADA 0040ca6c     jaccesswalker.obj
 0003:00000a80       ?theAccessInfoClassName@@3PADA 0040ca80     jaccesswalker.obj
 0003:00000ac0       ___security_cookie_complement 0040cac0     MSVCRT:gs_cookie.obj
 0003:00000ac4       ___security_cookie         0040cac4     MSVCRT:gs_cookie.obj
 0003:00000ac8       __fltused                  0040cac8     MSVCRT:fltused.obj
 0003:00000acc       ___scrt_native_dllmain_reason 0040cacc     MSVCRT:utility.obj
 0003:00000ad0       ___scrt_default_matherr    0040cad0     MSVCRT:matherr.obj
 0003:00000ae0       ___isa_enabled             0040cae0     MSVCRT:cpu_disp.obj
 0003:00000ae4       ___scrt_ucrt_dll_is_in_use 0040cae4     MSVCRT:ucrt_stubs.obj
 0003:00000ae8       ??_R0?AVbad_alloc@std@@@8  0040cae8     MSVCRT:throw_bad_alloc.obj
 0003:00000b04       ??_R0?AVexception@std@@@8  0040cb04     MSVCRT:throw_bad_alloc.obj
 0003:00000b20       ??_R0?AVbad_array_new_length@std@@@8 0040cb20     MSVCRT:throw_bad_alloc.obj
 0003:00000b48       ??_R0?AVtype_info@@@8      0040cb48     MSVCRT:std_type_info_static.obj
 0003:00000b60       _theAccessBridgeInitializedFlag 0040cb60     AccessBridgeCalls.obj
 0003:00000b68       ?_OptionsStorage@?1??__local_stdio_printf_options@@9@4_KA 0040cb68     AccessBridgeDebug.obj
 0003:00000c78       ?theFromJavaHelloMsgID@@3IA 0040cc78     AccessBridgeMessages.obj
 0003:00000c7c       ?theFromWindowsHelloMsgID@@3IA 0040cc7c     AccessBridgeMessages.obj
 0003:00000c80       ?g_LogStringCallback@@3P6GXPBD@ZA 0040cc80     AccessInfo.obj
 0003:00000cc8       ?ourHwnd@@3PAUHWND__@@A    0040ccc8     jaccesswalker.obj
 0003:00000ccc       ?topLevelWindow@@3PAUHWND__@@A 0040cccc     jaccesswalker.obj
 0003:00000cd0       ?logfile@@3PAU_iobuf@@A    0040ccd0     jaccesswalker.obj
 0003:00000cd4       ?popupMenu@@3PAUHMENU__@@A 0040ccd4     jaccesswalker.obj
 0003:00000cd8       ?theJaccesswalkerWindow@@3PAUHWND__@@A 0040ccd8     jaccesswalker.obj
 0003:00000cdc       ?theTreeControlWindow@@3PAUHWND__@@A 0040ccdc     jaccesswalker.obj
 0003:00000ce0       ?theInstance@@3PAUHINSTANCE__@@A 0040cce0     jaccesswalker.obj
 0003:00000ce4       ?theJaccesswalker@@3PAVJaccesswalker@@A 0040cce4     jaccesswalker.obj
 0003:00000ce8       ?theSelectedNode@@3PAVAccessibleNode@@A 0040cce8     jaccesswalker.obj
 0003:00000cec       ?thePopupNode@@3PAVAccessibleNode@@A 0040ccec     jaccesswalker.obj
 0003:00000cf0       ?theSelectedAccessibleContext@@3_JA 0040ccf0     jaccesswalker.obj
 0003:00000cf8       ?hwndTV@@3PAUHWND__@@A     0040ccf8     jaccesswalker.obj
 0003:0000101c       ___scrt_current_native_startup_state 0040d01c     MSVCRT:utility.obj
 0003:00001020       ___scrt_native_startup_lock 0040d020     MSVCRT:utility.obj
 0003:00001040       ?__type_info_root_node@@3U__type_info_node@@A 0040d040     MSVCRT:tncleanup.obj
 0003:00001048       ?_OptionsStorage@?1??__local_stdio_scanf_options@@9@4_KA 0040d048     MSVCRT:default_local_stdio_options.obj
 0003:00001050       ___scrt_debugger_hook_flag 0040d050     MSVCRT:utility_desktop.obj
 0003:00001054       ___isa_available           0040d054     MSVCRT:cpu_disp.obj
 0003:00001058       ___favor                   0040d058     MSVCRT:cpu_disp.obj
 0003:00001060       _theAccessBridge           0040d060     <common>
 0003:000011e4       _theAccessBridgeInstance   0040d1e4     <common>
 0003:000011e8       ___dyn_tls_dtor_callback   0040d1e8     <common>
 0003:000011ec       ___dyn_tls_init_callback   0040d1ec     <common>

 entry point at        0001:000065ec

 Static symbols

 0000:ffff0000       .debug$S                   00400000     vcruntime:VCRUNTIME140.dll
 0000:ffff0000       .debug$S                   00400000     vcruntime:VCRUNTIME140.dll
 0000:ffff0000       .debug$S                   00400000     vcruntime:VCRUNTIME140.dll
 0000:ffff0000       .debug$S                   00400000     vcruntime:VCRUNTIME140.dll
 0000:ffff0000       .debug$S                   00400000     vcruntime:VCRUNTIME140.dll
 0000:ffff0000       .debug$S                   00400000     vcruntime:VCRUNTIME140.dll
 0000:ffff0000       .debug$S                   00400000     vcruntime:VCRUNTIME140.dll
 0000:ffff0000       .debug$S                   00400000     vcruntime:VCRUNTIME140.dll
 0000:ffff0000       .debug$S                   00400000     vcruntime:VCRUNTIME140.dll
 0000:ffff0000       .debug$S                   00400000     vcruntime:VCRUNTIME140.dll
 0000:ffff0000       .debug$S                   00400000     ucrt:api-ms-win-crt-environment-l1-1-0.dll
 0000:ffff0000       .debug$S                   00400000     ucrt:api-ms-win-crt-heap-l1-1-0.dll
 0000:ffff0000       .debug$S                   00400000     ucrt:api-ms-win-crt-heap-l1-1-0.dll
 0000:ffff0000       .debug$S                   00400000     ucrt:api-ms-win-crt-heap-l1-1-0.dll
 0000:ffff0000       .debug$S                   00400000     ucrt:api-ms-win-crt-heap-l1-1-0.dll
 0000:ffff0000       .debug$S                   00400000     ucrt:api-ms-win-crt-locale-l1-1-0.dll
 0000:ffff0000       .debug$S                   00400000     ucrt:api-ms-win-crt-math-l1-1-0.dll
 0000:ffff0000       .debug$S                   00400000     ucrt:api-ms-win-crt-runtime-l1-1-0.dll
 0000:ffff0000       .debug$S                   00400000     ucrt:api-ms-win-crt-runtime-l1-1-0.dll
 0000:ffff0000       .debug$S                   00400000     ucrt:api-ms-win-crt-runtime-l1-1-0.dll
 0000:ffff0000       .debug$S                   00400000     ucrt:api-ms-win-crt-runtime-l1-1-0.dll
 0000:ffff0000       .debug$S                   00400000     ucrt:api-ms-win-crt-runtime-l1-1-0.dll
 0000:ffff0000       .debug$S                   00400000     ucrt:api-ms-win-crt-runtime-l1-1-0.dll
 0000:ffff0000       .debug$S                   00400000     ucrt:api-ms-win-crt-runtime-l1-1-0.dll
 0000:ffff0000       .debug$S                   00400000     ucrt:api-ms-win-crt-runtime-l1-1-0.dll
 0000:ffff0000       .debug$S                   00400000     ucrt:api-ms-win-crt-runtime-l1-1-0.dll
 0000:ffff0000       .debug$S                   00400000     ucrt:api-ms-win-crt-runtime-l1-1-0.dll
 0000:ffff0000       .debug$S                   00400000     ucrt:api-ms-win-crt-runtime-l1-1-0.dll
 0000:ffff0000       .debug$S                   00400000     ucrt:api-ms-win-crt-runtime-l1-1-0.dll
 0000:ffff0000       .debug$S                   00400000     ucrt:api-ms-win-crt-runtime-l1-1-0.dll
 0000:ffff0000       .debug$S                   00400000     ucrt:api-ms-win-crt-runtime-l1-1-0.dll
 0000:ffff0000       .debug$S                   00400000     ucrt:api-ms-win-crt-runtime-l1-1-0.dll
 0000:ffff0000       .debug$S                   00400000     ucrt:api-ms-win-crt-runtime-l1-1-0.dll
 0000:ffff0000       .debug$S                   00400000     ucrt:api-ms-win-crt-runtime-l1-1-0.dll
 0000:ffff0000       .debug$S                   00400000     ucrt:api-ms-win-crt-runtime-l1-1-0.dll
 0000:ffff0000       .debug$S                   00400000     ucrt:api-ms-win-crt-runtime-l1-1-0.dll
 0000:ffff0000       .debug$S                   00400000     ucrt:api-ms-win-crt-runtime-l1-1-0.dll
 0000:ffff0000       .debug$S                   00400000     ucrt:api-ms-win-crt-stdio-l1-1-0.dll
 0000:ffff0000       .debug$S                   00400000     ucrt:api-ms-win-crt-stdio-l1-1-0.dll
 0000:ffff0000       .debug$S                   00400000     ucrt:api-ms-win-crt-stdio-l1-1-0.dll
 0000:ffff0000       .debug$S                   00400000     ucrt:api-ms-win-crt-stdio-l1-1-0.dll
 0000:ffff0000       .debug$S                   00400000     ucrt:api-ms-win-crt-stdio-l1-1-0.dll
 0000:ffff0000       .debug$S                   00400000     ucrt:api-ms-win-crt-stdio-l1-1-0.dll
 0000:ffff0000       .debug$S                   00400000     ucrt:api-ms-win-crt-stdio-l1-1-0.dll
 0000:ffff0000       .debug$S                   00400000     ucrt:api-ms-win-crt-stdio-l1-1-0.dll
 0000:ffff0000       .debug$S                   00400000     ucrt:api-ms-win-crt-stdio-l1-1-0.dll
 0000:ffff0000       .debug$S                   00400000     ucrt:api-ms-win-crt-string-l1-1-0.dll
 0000:ffff0000       .debug$S                   00400000     ucrt:api-ms-win-crt-string-l1-1-0.dll
 0000:ffff0000       .debug$S                   00400000     ucrt:api-ms-win-crt-string-l1-1-0.dll
 0000:ffff0000       .debug$S                   00400000     ucrt:api-ms-win-crt-string-l1-1-0.dll
 0000:ffff0000       .debug$S                   00400000     ucrt:api-ms-win-crt-string-l1-1-0.dll
 0000:ffff0000       .debug$S                   00400000     ucrt:api-ms-win-crt-string-l1-1-0.dll
 0000:ffff0000       .debug$S                   00400000     ucrt:api-ms-win-crt-time-l1-1-0.dll
 0000:ffff0000       .debug$S                   00400000     ucrt:api-ms-win-crt-time-l1-1-0.dll
 0000:ffff0000       .debug$S                   00400000     ucrt:api-ms-win-crt-time-l1-1-0.dll
 0000:ffff0000       .debug$S                   00400000     comctl32:COMCTL32.dll
 0000:ffff0000       .debug$S                   00400000     gdi32:GDI32.dll
 0000:ffff0000       .debug$S                   00400000     kernel32:KERNEL32.dll
 0000:ffff0000       .debug$S                   00400000     kernel32:KERNEL32.dll
 0000:ffff0000       .debug$S                   00400000     kernel32:KERNEL32.dll
 0000:ffff0000       .debug$S                   00400000     kernel32:KERNEL32.dll
 0000:ffff0000       .debug$S                   00400000     kernel32:KERNEL32.dll
 0000:ffff0000       .debug$S                   00400000     kernel32:KERNEL32.dll
 0000:ffff0000       .debug$S                   00400000     kernel32:KERNEL32.dll
 0000:ffff0000       .debug$S                   00400000     kernel32:KERNEL32.dll
 0000:ffff0000       .debug$S                   00400000     kernel32:KERNEL32.dll
 0000:ffff0000       .debug$S                   00400000     kernel32:KERNEL32.dll
 0000:ffff0000       .debug$S                   00400000     kernel32:KERNEL32.dll
 0000:ffff0000       .debug$S                   00400000     kernel32:KERNEL32.dll
 0000:ffff0000       .debug$S                   00400000     kernel32:KERNEL32.dll
 0000:ffff0000       .debug$S                   00400000     kernel32:KERNEL32.dll
 0000:ffff0000       .debug$S                   00400000     kernel32:KERNEL32.dll
 0000:ffff0000       .debug$S                   00400000     kernel32:KERNEL32.dll
 0000:ffff0000       .debug$S                   00400000     kernel32:KERNEL32.dll
 0000:ffff0000       .debug$S                   00400000     kernel32:KERNEL32.dll
 0000:ffff0000       .debug$S                   00400000     kernel32:KERNEL32.dll
 0000:ffff0000       .debug$S                   00400000     user32:USER32.dll
 0000:ffff0000       .debug$S                   00400000     user32:USER32.dll
 0000:ffff0000       .debug$S                   00400000     user32:USER32.dll
 0000:ffff0000       .debug$S                   00400000     user32:USER32.dll
 0000:ffff0000       .debug$S                   00400000     user32:USER32.dll
 0000:ffff0000       .debug$S                   00400000     user32:USER32.dll
 0000:ffff0000       .debug$S                   00400000     user32:USER32.dll
 0000:ffff0000       .debug$S                   00400000     user32:USER32.dll
 0000:ffff0000       .debug$S                   00400000     user32:USER32.dll
 0000:ffff0000       .debug$S                   00400000     user32:USER32.dll
 0000:ffff0000       .debug$S                   00400000     user32:USER32.dll
 0000:ffff0000       .debug$S                   00400000     user32:USER32.dll
 0000:ffff0000       .debug$S                   00400000     user32:USER32.dll
 0000:ffff0000       .debug$S                   00400000     user32:USER32.dll
 0000:ffff0000       .debug$S                   00400000     user32:USER32.dll
 0000:ffff0000       .debug$S                   00400000     user32:USER32.dll
 0000:ffff0000       .debug$S                   00400000     user32:USER32.dll
 0000:ffff0000       .debug$S                   00400000     user32:USER32.dll
 0000:ffff0000       .debug$S                   00400000     user32:USER32.dll
 0000:ffff0000       .debug$S                   00400000     user32:USER32.dll
 0000:ffff0000       .debug$S                   00400000     user32:USER32.dll
 0000:ffff0000       .debug$S                   00400000     user32:USER32.dll
 0000:ffff0000       .debug$S                   00400000     user32:USER32.dll
 0000:ffff0000       .debug$S                   00400000     user32:USER32.dll
 0000:ffff0000       .debug$S                   00400000     user32:USER32.dll
 0000:ffff0000       .debug$S                   00400000     user32:USER32.dll
 0000:ffff0000       .debug$S                   00400000     user32:USER32.dll
 0000:ffff0000       .debug$S                   00400000     user32:USER32.dll
 0001:00004990       _localtime                 00405990 f   AccessInfo.obj
 0001:000049b0       _time                      004059b0 f   AccessInfo.obj
 0001:0000556c       $LN26                      0040656c     jaccesswalker.obj
 0001:00005580       $LN25                      00406580     jaccesswalker.obj
 0001:000062c0       $$000000                   004072c0     MSVCRT:ulldiv.obj
 0001:00006340       $$000000                   00407340     MSVCRT:chkstk.obj
 0001:000063ab       ?pre_c_initialization@@YAHXZ 004073ab f   MSVCRT:exe_winmain.obj
 0001:00006456       ?post_pgo_initialization@@YAHXZ 00407456 f   MSVCRT:exe_winmain.obj
 0001:0000645e       ?pre_cpp_initialization@@YAXXZ 0040745e f   MSVCRT:exe_winmain.obj
 0001:00006470       ?__scrt_common_main_seh@@YAHXZ 00407470 f   MSVCRT:exe_winmain.obj
 0001:00006712       ?find_pe_section@@YAPAU_IMAGE_SECTION_HEADER@@QAEI@Z 00407712 f   MSVCRT:utility.obj
 0001:00006963       ___get_entropy             00407963 f   MSVCRT:gs_support.obj
 0001:00006cd0       $$000000                   00407cd0     MSVCRT:sehprolg4.obj
 0001:000070c0       __unwindfunclet$?addComponentNodes@Jaccesswalker@@QAEXJ_JPAVAccessibleNode@@PAUHWND__@@PAU_TREEITEM@@2@Z$0 004080c0 f   jaccesswalker.obj
 0001:000070da       __ehhandler$?addComponentNodes@Jaccesswalker@@QAEXJ_JPAVAccessibleNode@@PAUHWND__@@PAU_TREEITEM@@2@Z 004080da f   jaccesswalker.obj
 0002:000001cc       ?pre_cpp_initializer@@3P6AXXZA 004091cc     MSVCRT:exe_winmain.obj
 0002:000001d8       ?pre_c_initializer@@3P6AHXZA 004091d8     MSVCRT:exe_winmain.obj
 0002:000001dc       ?post_pgo_initializer@@3P6AHXZA 004091dc     MSVCRT:exe_winmain.obj
 0002:000001f8       $SG43602                   004091f8     AccessBridgeDebug.obj
 0002:00000214       $SG43604                   00409214     AccessBridgeDebug.obj
 0002:0000021c       $SG43605                   0040921c     AccessBridgeDebug.obj
 0002:00000220       $SG43607                   00409220     AccessBridgeDebug.obj
 0002:00000228       $SG43608                   00409228     AccessBridgeDebug.obj
 0002:00000240       $SG43635                   00409240     AccessBridgeDebug.obj
 0002:0000025c       $SG43636                   0040925c     AccessBridgeDebug.obj
 0002:00000268       $SG43638                   00409268     AccessBridgeDebug.obj
 0002:0000026c       $SG43680                   0040926c     AccessBridgeDebug.obj
 0002:00000274       $SG43681                   00409274     AccessBridgeDebug.obj
 0002:00000278       $SG43697                   00409278     AccessBridgeDebug.obj
 0002:00000280       $SG43698                   00409280     AccessBridgeDebug.obj
 0002:00000284       $SG43740                   00409284     AccessBridgeDebug.obj
 0002:0000028c       $SG43741                   0040928c     AccessBridgeDebug.obj
 0002:00000290       $SG43757                   00409290     AccessBridgeDebug.obj
 0002:00000298       $SG43758                   00409298     AccessBridgeDebug.obj
 0002:0000029c       $SG38458                   0040929c     AccessBridgeMessages.obj
 0002:000002b8       $SG38459                   004092b8     AccessBridgeMessages.obj
 0002:000002d8       $SG47878                   004092d8     AccessInfo.obj
 0002:000002dc       $SG47880                   004092dc     AccessInfo.obj
 0002:000002e0       $SG47883                   004092e0     AccessInfo.obj
 0002:000002ec       $SG47928                   004092ec     AccessInfo.obj
 0002:00000318       $SG47929                   00409318     AccessInfo.obj
 0002:0000031c       $SG47930                   0040931c     AccessInfo.obj
 0002:00000320       $SG47948                   00409320     AccessInfo.obj
 0002:00000324       $SG48090                   00409324     AccessInfo.obj
 0002:0000034c       $SG48091                   0040934c     AccessInfo.obj
 0002:00000364       $SG48092                   00409364     AccessInfo.obj
 0002:0000038c       $SG48093                   0040938c     AccessInfo.obj
 0002:000003b8       $SG48094                   004093b8     AccessInfo.obj
 0002:000003e4       $SG48095                   004093e4     AccessInfo.obj
 0002:00000414       $SG48099                   00409414     AccessInfo.obj
 0002:00000440       $SG48100                   00409440     AccessInfo.obj
 0002:00000464       $SG48103                   00409464     AccessInfo.obj
 0002:00000480       $SG48104                   00409480     AccessInfo.obj
 0002:00000484       $SG48105                   00409484     AccessInfo.obj
 0002:00000498       $SG48108                   00409498     AccessInfo.obj
 0002:000004bc       $SG48109                   004094bc     AccessInfo.obj
 0002:000004d8       $SG48110                   004094d8     AccessInfo.obj
 0002:000004f0       $SG48111                   004094f0     AccessInfo.obj
 0002:00000504       $SG48112                   00409504     AccessInfo.obj
 0002:00000528       $SG48113                   00409528     AccessInfo.obj
 0002:0000053c       $SG48114                   0040953c     AccessInfo.obj
 0002:00000560       $SG48115                   00409560     AccessInfo.obj
 0002:0000057c       $SG48116                   0040957c     AccessInfo.obj
 0002:00000598       $SG48117                   00409598     AccessInfo.obj
 0002:000005c4       $SG48120                   004095c4     AccessInfo.obj
 0002:000005e8       $SG48123                   004095e8     AccessInfo.obj
 0002:00000628       $SG48126                   00409628     AccessInfo.obj
 0002:0000064c       $SG48127                   0040964c     AccessInfo.obj
 0002:00000670       $SG48128                   00409670     AccessInfo.obj
 0002:00000694       $SG48131                   00409694     AccessInfo.obj
 0002:000006a4       $SG48134                   004096a4     AccessInfo.obj
 0002:000006d8       $SG48135                   004096d8     AccessInfo.obj
 0002:000006f0       $SG48138                   004096f0     AccessInfo.obj
 0002:00000714       $SG48139                   00409714     AccessInfo.obj
 0002:00000734       $SG48140                   00409734     AccessInfo.obj
 0002:0000074c       $SG48143                   0040974c     AccessInfo.obj
 0002:00000774       $SG48144                   00409774     AccessInfo.obj
 0002:0000079c       $SG48148                   0040979c     AccessInfo.obj
 0002:000007c0       $SG48152                   004097c0     AccessInfo.obj
 0002:000007e4       $SG48153                   004097e4     AccessInfo.obj
 0002:00000804       $SG48154                   00409804     AccessInfo.obj
 0002:00000824       $SG48156                   00409824     AccessInfo.obj
 0002:0000084c       $SG48158                   0040984c     AccessInfo.obj
 0002:00000868       $SG48161                   00409868     AccessInfo.obj
 0002:000008ac       $SG48164                   004098ac     AccessInfo.obj
 0002:000008e8       $SG48167                   004098e8     AccessInfo.obj
 0002:0000090c       $SG48168                   0040990c     AccessInfo.obj
 0002:0000092c       $SG48169                   0040992c     AccessInfo.obj
 0002:0000094c       $SG48170                   0040994c     AccessInfo.obj
 0002:00000978       $SG48172                   00409978     AccessInfo.obj
 0002:00000998       $SG48173                   00409998     AccessInfo.obj
 0002:000009bc       $SG48174                   004099bc     AccessInfo.obj
 0002:000009e0       $SG48175                   004099e0     AccessInfo.obj
 0002:00000a04       $SG48177                   00409a04     AccessInfo.obj
 0002:00000a20       $SG48178                   00409a20     AccessInfo.obj
 0002:00000a3c       $SG48179                   00409a3c     AccessInfo.obj
 0002:00000a5c       $SG48180                   00409a5c     AccessInfo.obj
 0002:00000a78       $SG48181                   00409a78     AccessInfo.obj
 0002:00000a90       $SG48183                   00409a90     AccessInfo.obj
 0002:00000aac       $SG48184                   00409aac     AccessInfo.obj
 0002:00000acc       $SG48185                   00409acc     AccessInfo.obj
 0002:00000ae8       $SG48188                   00409ae8     AccessInfo.obj
 0002:00000b0c       $SG48190                   00409b0c     AccessInfo.obj
 0002:00000b34       $SG48191                   00409b34     AccessInfo.obj
 0002:00000b54       $SG48192                   00409b54     AccessInfo.obj
 0002:00000b70       $SG48193                   00409b70     AccessInfo.obj
 0002:00000b94       $SG48196                   00409b94     AccessInfo.obj
 0002:00000bc0       $SG48199                   00409bc0     AccessInfo.obj
 0002:00000be4       $SG48200                   00409be4     AccessInfo.obj
 0002:00000c04       $SG48201                   00409c04     AccessInfo.obj
 0002:00000c24       $SG48203                   00409c24     AccessInfo.obj
 0002:00000c48       $SG48205                   00409c48     AccessInfo.obj
 0002:00000c64       $SG48207                   00409c64     AccessInfo.obj
 0002:00000c80       $SG48209                   00409c80     AccessInfo.obj
 0002:00000c9c       $SG48213                   00409c9c     AccessInfo.obj
 0002:00000cc4       $SG48214                   00409cc4     AccessInfo.obj
 0002:00000ce0       $SG48215                   00409ce0     AccessInfo.obj
 0002:00000d04       $SG48216                   00409d04     AccessInfo.obj
 0002:00000d28       $SG48217                   00409d28     AccessInfo.obj
 0002:00000d4c       $SG48218                   00409d4c     AccessInfo.obj
 0002:00000d68       $SG48219                   00409d68     AccessInfo.obj
 0002:00000d88       $SG48222                   00409d88     AccessInfo.obj
 0002:00000db4       $SG48223                   00409db4     AccessInfo.obj
 0002:00000de0       $SG48224                   00409de0     AccessInfo.obj
 0002:00000df4       $SG48225                   00409df4     AccessInfo.obj
 0002:00000e0c       $SG48226                   00409e0c     AccessInfo.obj
 0002:00000e28       $SG48227                   00409e28     AccessInfo.obj
 0002:00000e40       $SG48230                   00409e40     AccessInfo.obj
 0002:00000e84       $SG48233                   00409e84     AccessInfo.obj
 0002:00000ea8       $SG48234                   00409ea8     AccessInfo.obj
 0002:00000ebc       $SG48235                   00409ebc     AccessInfo.obj
 0002:00000ed0       $SG48238                   00409ed0     AccessInfo.obj
 0002:00000f00       $SG48239                   00409f00     AccessInfo.obj
 0002:00000f28       $SG48240                   00409f28     AccessInfo.obj
 0002:00000f4c       $SG48241                   00409f4c     AccessInfo.obj
 0002:00000f74       $SG48242                   00409f74     AccessInfo.obj
 0002:00000f94       $SG48245                   00409f94     AccessInfo.obj
 0002:00000fc8       $SG48246                   00409fc8     AccessInfo.obj
 0002:00000fe0       $SG48247                   00409fe0     AccessInfo.obj
 0002:00000fe4       $SG48250                   00409fe4     AccessInfo.obj
 0002:00001010       $SG48251                   0040a010     AccessInfo.obj
 0002:00001034       $SG48252                   0040a034     AccessInfo.obj
 0002:00001048       $SG48253                   0040a048     AccessInfo.obj
 0002:00001060       $SG48254                   0040a060     AccessInfo.obj
 0002:0000107c       $SG48255                   0040a07c     AccessInfo.obj
 0002:00001094       $SG48258                   0040a094     AccessInfo.obj
 0002:000010c0       $SG48261                   0040a0c0     AccessInfo.obj
 0002:000010e4       $SG48262                   0040a0e4     AccessInfo.obj
 0002:000010f8       $SG48263                   0040a0f8     AccessInfo.obj
 0002:0000110c       $SG48265                   0040a10c     AccessInfo.obj
 0002:00001130       $SG48267                   0040a130     AccessInfo.obj
 0002:00001158       $SG48268                   0040a158     AccessInfo.obj
 0002:00001178       $SG48269                   0040a178     AccessInfo.obj
 0002:00001190       $SG48271                   0040a190     AccessInfo.obj
 0002:000011b4       $SG48272                   0040a1b4     AccessInfo.obj
 0002:000011d4       $SG48273                   0040a1d4     AccessInfo.obj
 0002:000011f0       $SG48274                   0040a1f0     AccessInfo.obj
 0002:00001214       $SG48276                   0040a214     AccessInfo.obj
 0002:00001250       $SG48279                   0040a250     AccessInfo.obj
 0002:00001270       $SG48281                   0040a270     AccessInfo.obj
 0002:0000128c       $SG48282                   0040a28c     AccessInfo.obj
 0002:000012a4       $SG48283                   0040a2a4     AccessInfo.obj
 0002:000012c0       $SG48285                   0040a2c0     AccessInfo.obj
 0002:000012c8       $SG48286                   0040a2c8     AccessInfo.obj
 0002:000012d4       $SG48287                   0040a2d4     AccessInfo.obj
 0002:000012f4       $SG48288                   0040a2f4     AccessInfo.obj
 0002:000012fc       $SG48289                   0040a2fc     AccessInfo.obj
 0002:00001308       $SG48290                   0040a308     AccessInfo.obj
 0002:00001310       $SG48291                   0040a310     AccessInfo.obj
 0002:0000131c       $SG48292                   0040a31c     AccessInfo.obj
 0002:0000132c       $SG48293                   0040a32c     AccessInfo.obj
 0002:00001334       $SG48294                   0040a334     AccessInfo.obj
 0002:00001344       $SG48295                   0040a344     AccessInfo.obj
 0002:00001358       $SG48296                   0040a358     AccessInfo.obj
 0002:00001360       $SG48297                   0040a360     AccessInfo.obj
 0002:0000136c       $SG48298                   0040a36c     AccessInfo.obj
 0002:0000137c       $SG48299                   0040a37c     AccessInfo.obj
 0002:00001384       $SG48300                   0040a384     AccessInfo.obj
 0002:00001390       $SG48301                   0040a390     AccessInfo.obj
 0002:000013a0       $SG48302                   0040a3a0     AccessInfo.obj
 0002:000013a8       $SG48303                   0040a3a8     AccessInfo.obj
 0002:000013cc       $SG48304                   0040a3cc     AccessInfo.obj
 0002:000013f0       $SG48305                   0040a3f0     AccessInfo.obj
 0002:0000140c       $SG48306                   0040a40c     AccessInfo.obj
 0002:00001428       $SG48307                   0040a428     AccessInfo.obj
 0002:0000144c       $SG48308                   0040a44c     AccessInfo.obj
 0002:00001468       $SG48309                   0040a468     AccessInfo.obj
 0002:00001484       $SG48310                   0040a484     AccessInfo.obj
 0002:000014a0       $SG48311                   0040a4a0     AccessInfo.obj
 0002:000014bc       $SG48312                   0040a4bc     AccessInfo.obj
 0002:000014d8       $SG48313                   0040a4d8     AccessInfo.obj
 0002:00001500       $SG48316                   0040a500     AccessInfo.obj
 0002:00001520       $SG48317                   0040a520     AccessInfo.obj
 0002:0000154c       $SG48318                   0040a54c     AccessInfo.obj
 0002:00001568       $SG48320                   0040a568     AccessInfo.obj
 0002:000015a0       $SG48322                   0040a5a0     AccessInfo.obj
 0002:000015dc       $SG48325                   0040a5dc     AccessInfo.obj
 0002:000015fc       $SG48327                   0040a5fc     AccessInfo.obj
 0002:00001618       $SG48328                   0040a618     AccessInfo.obj
 0002:00001630       $SG48329                   0040a630     AccessInfo.obj
 0002:0000164c       $SG48331                   0040a64c     AccessInfo.obj
 0002:00001654       $SG48332                   0040a654     AccessInfo.obj
 0002:00001660       $SG48333                   0040a660     AccessInfo.obj
 0002:00001680       $SG48334                   0040a680     AccessInfo.obj
 0002:00001688       $SG48335                   0040a688     AccessInfo.obj
 0002:00001694       $SG48336                   0040a694     AccessInfo.obj
 0002:0000169c       $SG48337                   0040a69c     AccessInfo.obj
 0002:000016a8       $SG48338                   0040a6a8     AccessInfo.obj
 0002:000016b8       $SG48339                   0040a6b8     AccessInfo.obj
 0002:000016c0       $SG48340                   0040a6c0     AccessInfo.obj
 0002:000016d0       $SG48341                   0040a6d0     AccessInfo.obj
 0002:000016e4       $SG48342                   0040a6e4     AccessInfo.obj
 0002:000016ec       $SG48343                   0040a6ec     AccessInfo.obj
 0002:000016f8       $SG48344                   0040a6f8     AccessInfo.obj
 0002:00001708       $SG48345                   0040a708     AccessInfo.obj
 0002:00001710       $SG48346                   0040a710     AccessInfo.obj
 0002:0000171c       $SG48347                   0040a71c     AccessInfo.obj
 0002:0000172c       $SG48348                   0040a72c     AccessInfo.obj
 0002:00001734       $SG48349                   0040a734     AccessInfo.obj
 0002:00001758       $SG48350                   0040a758     AccessInfo.obj
 0002:0000177c       $SG48351                   0040a77c     AccessInfo.obj
 0002:00001798       $SG48352                   0040a798     AccessInfo.obj
 0002:000017b4       $SG48353                   0040a7b4     AccessInfo.obj
 0002:000017d8       $SG48354                   0040a7d8     AccessInfo.obj
 0002:000017f4       $SG48355                   0040a7f4     AccessInfo.obj
 0002:00001810       $SG48356                   0040a810     AccessInfo.obj
 0002:0000182c       $SG48357                   0040a82c     AccessInfo.obj
 0002:00001848       $SG48358                   0040a848     AccessInfo.obj
 0002:00001864       $SG48359                   0040a864     AccessInfo.obj
 0002:0000188c       $SG48362                   0040a88c     AccessInfo.obj
 0002:000018ac       $SG48363                   0040a8ac     AccessInfo.obj
 0002:000018d8       $SG55727                   0040a8d8     jaccesswalker.obj
 0002:000018da       $SG55775                   0040a8da     jaccesswalker.obj
 0002:000018db       $SG55849                   0040a8db     jaccesswalker.obj
 0002:000018dc       $SG55728                   0040a8dc     jaccesswalker.obj
 0002:000018ee       $SG55952                   0040a8ee     jaccesswalker.obj
 0002:000018f0       $SG55729                   0040a8f0     jaccesswalker.obj
 0002:00001910       $SG55815                   0040a910     jaccesswalker.obj
 0002:0000191c       $SG55850                   0040a91c     jaccesswalker.obj
 0002:00001924       $SG55878                   0040a924     jaccesswalker.obj
 0002:0000192c       $SG55879                   0040a92c     jaccesswalker.obj
 0002:00001944       $SG55902                   0040a944     jaccesswalker.obj
 0002:00001950       $SG55909                   0040a950     jaccesswalker.obj
 0002:0000195c       $SG55913                   0040a95c     jaccesswalker.obj
 0002:00001968       $SG55915                   0040a968     jaccesswalker.obj
 0002:00001974       $SG55918                   0040a974     jaccesswalker.obj
 0002:00001980       $SG55920                   0040a980     jaccesswalker.obj
 0002:00001990       $SG55922                   0040a990     jaccesswalker.obj
 0002:0000199c       $SG55927                   0040a99c     jaccesswalker.obj
 0002:000019a8       $SG55929                   0040a9a8     jaccesswalker.obj
 0002:000019b4       $SG55932                   0040a9b4     jaccesswalker.obj
 0002:000019c0       $SG55953                   0040a9c0     jaccesswalker.obj
 0002:000019d0       $SG55999                   0040a9d0     jaccesswalker.obj
 0002:000019d4       $SG56000                   0040a9d4     jaccesswalker.obj
 0002:000019d8       $SG56001                   0040a9d8     jaccesswalker.obj
 0002:000019e4       $SG56032                   0040a9e4     jaccesswalker.obj
 0002:00001a00       $SG56002                   0040aa00     jaccesswalker.obj
 0002:00001a40       $SG56034                   0040aa40     jaccesswalker.obj
 0002:00001a5c       _GS_ExceptionPointers      0040aa5c     MSVCRT:gs_report.obj
 0002:00002030       __unwindtable$?addComponentNodes@Jaccesswalker@@QAEXJ_JPAVAccessibleNode@@PAUHWND__@@PAU_TREEITEM@@2@Z 0040b030     jaccesswalker.obj
 0002:00002038       __ehfuncinfo$?addComponentNodes@Jaccesswalker@@QAEXJ_JPAVAccessibleNode@@PAUHWND__@@PAU_TREEITEM@@2@Z 0040b038     jaccesswalker.obj
 0002:00002060       __sehtable$?__scrt_common_main_seh@@YAHXZ 0040b060     MSVCRT:exe_winmain.obj
 0002:00002110       __sehtable$___scrt_is_nonwritable_in_current_image 0040b110     MSVCRT:utility.obj
 0002:00002420       .idata$6                   0040b420     comctl32:COMCTL32.dll
 0002:00002440       .idata$6                   0040b440     gdi32:GDI32.dll
 0002:00002614       .idata$6                   0040b614     user32:USER32.dll
 0002:000027ac       .idata$6                   0040b7ac     kernel32:KERNEL32.dll
 0002:0000287a       .idata$6                   0040b87a     vcruntime:VCRUNTIME140.dll
 0002:00002b3a       .idata$6                   0040bb3a     ucrt:api-ms-win-crt-string-l1-1-0.dll
 0002:00002b5c       .idata$6                   0040bb5c     ucrt:api-ms-win-crt-stdio-l1-1-0.dll
 0002:00002b7c       .idata$6                   0040bb7c     ucrt:api-ms-win-crt-environment-l1-1-0.dll
 0002:00002ba2       .idata$6                   0040bba2     ucrt:api-ms-win-crt-time-l1-1-0.dll
 0002:00002bc2       .idata$6                   0040bbc2     ucrt:api-ms-win-crt-heap-l1-1-0.dll
 0002:00002be2       .idata$6                   0040bbe2     ucrt:api-ms-win-crt-runtime-l1-1-0.dll
 0002:00002c04       .idata$6                   0040bc04     ucrt:api-ms-win-crt-math-l1-1-0.dll
 0002:00002c24       .idata$6                   0040bc24     ucrt:api-ms-win-crt-locale-l1-1-0.dll
 0003:00000000       $SG46443                   0040c000     AccessBridgeCalls.obj
 0003:00000018       $SG46447                   0040c018     AccessBridgeCalls.obj
 0003:00000024       $SG46449                   0040c024     AccessBridgeCalls.obj
 0003:00000038       $SG46451                   0040c038     AccessBridgeCalls.obj
 0003:0000004c       $SG46453                   0040c04c     AccessBridgeCalls.obj
 0003:0000005c       $SG46455                   0040c05c     AccessBridgeCalls.obj
 0003:00000070       $SG46457                   0040c070     AccessBridgeCalls.obj
 0003:00000084       $SG46459                   0040c084     AccessBridgeCalls.obj
 0003:00000098       $SG46461                   0040c098     AccessBridgeCalls.obj
 0003:000000ac       $SG46463                   0040c0ac     AccessBridgeCalls.obj
 0003:000000c0       $SG46465                   0040c0c0     AccessBridgeCalls.obj
 0003:000000d4       $SG46467                   0040c0d4     AccessBridgeCalls.obj
 0003:000000e8       $SG46469                   0040c0e8     AccessBridgeCalls.obj
 0003:000000fc       $SG46471                   0040c0fc     AccessBridgeCalls.obj
 0003:00000110       $SG46473                   0040c110     AccessBridgeCalls.obj
 0003:00000128       $SG46475                   0040c128     AccessBridgeCalls.obj
 0003:0000014c       $SG46477                   0040c14c     AccessBridgeCalls.obj
 0003:0000016c       $SG46479                   0040c16c     AccessBridgeCalls.obj
 0003:00000184       $SG46481                   0040c184     AccessBridgeCalls.obj
 0003:000001a4       $SG46483                   0040c1a4     AccessBridgeCalls.obj
 0003:000001c0       $SG46485                   0040c1c0     AccessBridgeCalls.obj
 0003:000001dc       $SG46487                   0040c1dc     AccessBridgeCalls.obj
 0003:000001fc       $SG46489                   0040c1fc     AccessBridgeCalls.obj
 0003:00000214       $SG46491                   0040c214     AccessBridgeCalls.obj
 0003:00000230       $SG46493                   0040c230     AccessBridgeCalls.obj
 0003:00000250       $SG46495                   0040c250     AccessBridgeCalls.obj
 0003:0000026c       $SG46497                   0040c26c     AccessBridgeCalls.obj
 0003:00000290       $SG46499                   0040c290     AccessBridgeCalls.obj
 0003:000002b0       $SG46501                   0040c2b0     AccessBridgeCalls.obj
 0003:000002c4       $SG46503                   0040c2c4     AccessBridgeCalls.obj
 0003:000002d4       $SG46505                   0040c2d4     AccessBridgeCalls.obj
 0003:000002e4       $SG46507                   0040c2e4     AccessBridgeCalls.obj
 0003:000002f4       $SG46509                   0040c2f4     AccessBridgeCalls.obj
 0003:00000314       $SG46511                   0040c314     AccessBridgeCalls.obj
 0003:00000334       $SG46513                   0040c334     AccessBridgeCalls.obj
 0003:0000034c       $SG46515                   0040c34c     AccessBridgeCalls.obj
 0003:0000036c       $SG46517                   0040c36c     AccessBridgeCalls.obj
 0003:00000388       $SG46519                   0040c388     AccessBridgeCalls.obj
 0003:000003a8       $SG46521                   0040c3a8     AccessBridgeCalls.obj
 0003:000003c8       $SG46523                   0040c3c8     AccessBridgeCalls.obj
 0003:000003e0       $SG46525                   0040c3e0     AccessBridgeCalls.obj
 0003:000003fc       $SG46527                   0040c3fc     AccessBridgeCalls.obj
 0003:00000418       $SG46529                   0040c418     AccessBridgeCalls.obj
 0003:00000438       $SG46531                   0040c438     AccessBridgeCalls.obj
 0003:0000045c       $SG46533                   0040c45c     AccessBridgeCalls.obj
 0003:00000480       $SG46535                   0040c480     AccessBridgeCalls.obj
 0003:000004a4       $SG46537                   0040c4a4     AccessBridgeCalls.obj
 0003:000004c4       $SG46539                   0040c4c4     AccessBridgeCalls.obj
 0003:000004e4       $SG46541                   0040c4e4     AccessBridgeCalls.obj
 0003:0000050c       $SG46543                   0040c50c     AccessBridgeCalls.obj
 0003:0000052c       $SG46545                   0040c52c     AccessBridgeCalls.obj
 0003:00000550       $SG46547                   0040c550     AccessBridgeCalls.obj
 0003:00000568       $SG46549                   0040c568     AccessBridgeCalls.obj
 0003:00000584       $SG46551                   0040c584     AccessBridgeCalls.obj
 0003:0000059c       $SG46553                   0040c59c     AccessBridgeCalls.obj
 0003:000005b8       $SG46555                   0040c5b8     AccessBridgeCalls.obj
 0003:000005d0       $SG46557                   0040c5d0     AccessBridgeCalls.obj
 0003:000005ec       $SG46559                   0040c5ec     AccessBridgeCalls.obj
 0003:00000608       $SG46561                   0040c608     AccessBridgeCalls.obj
 0003:00000624       $SG46563                   0040c624     AccessBridgeCalls.obj
 0003:00000644       $SG46565                   0040c644     AccessBridgeCalls.obj
 0003:0000065c       $SG46567                   0040c65c     AccessBridgeCalls.obj
 0003:00000678       $SG46569                   0040c678     AccessBridgeCalls.obj
 0003:0000068c       $SG46571                   0040c68c     AccessBridgeCalls.obj
 0003:000006a4       $SG46573                   0040c6a4     AccessBridgeCalls.obj
 0003:000006b8       $SG46575                   0040c6b8     AccessBridgeCalls.obj
 0003:000006d0       $SG46577                   0040c6d0     AccessBridgeCalls.obj
 0003:000006e8       $SG46579                   0040c6e8     AccessBridgeCalls.obj
 0003:00000708       $SG46581                   0040c708     AccessBridgeCalls.obj
 0003:00000724       $SG46583                   0040c724     AccessBridgeCalls.obj
 0003:0000073c       $SG46585                   0040c73c     AccessBridgeCalls.obj
 0003:00000758       $SG46587                   0040c758     AccessBridgeCalls.obj
 0003:00000770       $SG46589                   0040c770     AccessBridgeCalls.obj
 0003:00000798       $SG46591                   0040c798     AccessBridgeCalls.obj
 0003:000007c0       $SG46593                   0040c7c0     AccessBridgeCalls.obj
 0003:000007e8       $SG46595                   0040c7e8     AccessBridgeCalls.obj
 0003:0000080c       $SG46597                   0040c80c     AccessBridgeCalls.obj
 0003:00000830       $SG46599                   0040c830     AccessBridgeCalls.obj
 0003:00000854       $SG46601                   0040c854     AccessBridgeCalls.obj
 0003:0000087c       $SG46603                   0040c87c     AccessBridgeCalls.obj
 0003:000008a4       $SG46605                   0040c8a4     AccessBridgeCalls.obj
 0003:000008cc       $SG46607                   0040c8cc     AccessBridgeCalls.obj
 0003:000008f4       $SG46609                   0040c8f4     AccessBridgeCalls.obj
 0003:00000904       $SG46611                   0040c904     AccessBridgeCalls.obj
 0003:00000918       $SG46613                   0040c918     AccessBridgeCalls.obj
 0003:0000092c       $SG46615                   0040c92c     AccessBridgeCalls.obj
 0003:00000948       $SG46617                   0040c948     AccessBridgeCalls.obj
 0003:00000958       $SG46619                   0040c958     AccessBridgeCalls.obj
 0003:0000096c       $SG46621                   0040c96c     AccessBridgeCalls.obj
 0003:00000988       $SG46623                   0040c988     AccessBridgeCalls.obj
 0003:00000998       $SG46625                   0040c998     AccessBridgeCalls.obj
 0003:000009a8       $SG46627                   0040c9a8     AccessBridgeCalls.obj
 0003:000009c4       $SG46629                   0040c9c4     AccessBridgeCalls.obj
 0003:000009dc       $SG46631                   0040c9dc     AccessBridgeCalls.obj
 0003:000009f0       $SG46633                   0040c9f0     AccessBridgeCalls.obj
 0003:00000a04       $SG46635                   0040ca04     AccessBridgeCalls.obj
 0003:00000a18       $SG46637                   0040ca18     AccessBridgeCalls.obj
 0003:00000a2c       ?warning@?1??appendToBuffer@@YAHPADI0ZZ@4PADA 0040ca2c     AccessInfo.obj
 0003:00000a90       ?szAppName@?1???0Jaccesswalker@@QAE@H@Z@4PADA 0040ca90     jaccesswalker.obj
 0003:00000aa0       ?szMenuName@?1???0Jaccesswalker@@QAE@H@Z@4PADA 0040caa0     jaccesswalker.obj
 0003:00000b70       _logFP                     0040cb70     AccessBridgeDebug.obj
 0003:00000b78       ?retbuf@?1??printError@@9@4PADA 0040cb78     AccessBridgeDebug.obj
 0003:00000c88       ?datebuf@?1??getTimeAndDate@@YAPADXZ@4PADA 0040cc88     AccessInfo.obj
 0003:00000d00       _GS_ExceptionRecord        0040cd00     MSVCRT:gs_report.obj
 0003:00000d50       _GS_ContextRecord          0040cd50     MSVCRT:gs_report.obj
 0003:00001024       ?is_initialized_as_dll@@3_NA 0040d024     MSVCRT:utility.obj
 0003:00001025       ?module_local_atexit_table_initialized@@3_NA 0040d025     MSVCRT:utility.obj
 0003:00001028       ?module_local_atexit_table@@3U_onexit_table_t@@A 0040d028     MSVCRT:utility.obj
 0003:00001034       ?module_local_at_quick_exit_table@@3U_onexit_table_t@@A 0040d034     MSVCRT:utility.obj
 0004:000001d0       $R000000                   0040e1d0     jaccesswalker-32.exe.res
 0004:00000518       $R000348                   0040e518     jaccesswalker-32.exe.res
 0004:000005a8       $R0003D8                   0040e5a8     jaccesswalker-32.exe.res
 0004:00000638       $R000468                   0040e638     jaccesswalker-32.exe.res
 0004:000006d8       $R000508                   0040e6d8     jaccesswalker-32.exe.res
